:020000041100E9
:1030000070B500234025294C0120636101F0F8F9D7
:103010000223FE212800264A257401F077FA0028B1
:1030200035D10223FF21234A207C01F06FFA0028CA
:103030002DD1214BA2899A4226D1E3891F4A93427E
:103040000ED11F4B1F4963612368002B05D1002956
:1030500003D00C22200008F04BF901F045FA70BDB6
:10306000194A934201D00021EEE7184B184A1B6819
:10307000934205D9C02204212800920001F0C0FA31
:103080000F4B14496361DFE700232374EBE7CC2285
:103090003820AC219201207401F0B2FA0028F3D15B
:1030A0000D4B0E4963610E4BE381CDE7E462FF1FD8
:1030B000F062FF1FF262FF1F5959000083050000F4
:1030C0008142001188B80011821500002863FF1F9B
:1030D0008713000094B80011094300117CB8001157
:1030E000AAAAFFFFF7B5164B0192C318021D0020D4
:1030F000009388235B05D3181B685C1C1AD09CB214
:10310000402C18D88D781E0CAC466746CD782D0221
:103110003D43AE4206D1019800280ED110000C703C
:10312000240A4C7003249BB20733A343D218009B9C
:103130009A42DED3FEBD4432F9E71000FAE7C046FA
:10314000FC0F0000802213B503000324019189B213
:10315000520107319B18A14304305A1A88235B059A
:10316000C3181B68591C03D190429241104016BDF0
:1031700099B2402907D80B000733A343C0189042E7
:10318000ECD30020F3E74430F9E7134B134A1B68F4
:10319000126810B5FA24934201D81A00F824104B93
:1031A000E4021B689A4210D813000E4A12689A4231
:1031B0000ED3013307D1F823DB029C4203D10A4925
:1031C000054808F0FDF9200010BDFC24E402ECE7FE
:1031D000FE24E402F7E7C04600C0071100D0071143
:1031E00000E0071100F00711FFFFFF7FF0B59BB073
:1031F000150004900391402A00D9A0E006AB598045
:103200001A80FFF7C2FF0400042816D9002206A97D
:10321000FFF768FF052810D906AB1B88AB420CD11D
:10322000002D07D0514B2A000499C01808F040FA2D
:10323000002802D101201BB0F0BD06AB1D8020008C
:103240000699FFF77FFF041E7BD1069B0793FFF7CC
:103250009CFF80235B01C618802307001B039E424E
:1032600001D3F826F60288235B05F31801931B6847
:10327000013302D0019807F0ABFF3D49019808F0F7
:103280009FF93B1D0293331D05938822029B520533
:103290009B181B6808935A1C3CD044219AB2009199
:1032A000402A04D80320D11D814389B2009103999B
:1032B0001B0C8B4224D0402A22D80122300008A9BE
:1032C000FFF710FF021E1BD1380008A9FFF70AFF05
:1032D0000400042831D9009A059B9B1880225201D2
:1032E000B218934240D288235B05C118009A09A8FE
:1032F00008F00EFA1D4B009A09A9F01808F070F8B2
:10330000009A029B9446634402931A4B029AFB185C
:103310009A42BAD388235B05FC18216801980139C9
:1033200008F04EF9200007F053FF039A07AB5A80CC
:1033300030000799FFF706FF0400002C03D100209E
:1033400079E70428FBD988235B05E018069908F083
:1033500037F90323EA1C9A4300D16BE7034B049926
:10336000E01808F03DF865E70424ECE704000011DC
:10337000FFFFFF7FF80F0000F7B505001400402A9B
:1033800021D8002701AE71803780FFF7FEFE0428A8
:1033900016D93A003100FFF7A5FE042810D9368867
:1033A000BC420BD0BD4209D0221CB44200D9321C11
:1033B000064B92B2C118280008F0AAF930B2FEBD3F
:1033C000C04300B2FBE703204042F8E704000011CD
:1033D00037B5042204000D0001A81649FFF7CCFF01
:1033E000020004280BD1019BA34208D3AB4204D0B6
:1033F000104901A80195FFF7F9FE01203EBD0E4CD2
:1034000023682000019307F0E3FE019920000139B1
:10341000019108F0D5F880235B01E418074B9C422A
:10342000EED10422034901A80195FFF7DFFE002039
:10343000E4E7C0465555000000C007110000081120
:1034400030B589B007F0A4FE10226946254808F07F
:103450000FF9254B009A9A420ED1019B029A0F2B2D
:1034600033D8002101240698013B08D2002900D05E
:103470000292029B013331D10023029325E0551CB7
:10348000F2D102002100EFE710341022200004A93D
:1034900008F0EEF8029B013301D1069B02938823CA
:1034A00004995B05C918059B06981A03120B049131
:1034B0000592814203D02B4201D107F019FF019BF5
:1034C000013B0193019B002BDED1029B002B03D01B
:1034D000049304984168084709B030BDE025014CC9
:1034E0002D03EFE70000011150485936F7B50F4999
:1034F0000F4B0A6804001A4084235B0013430B60DF
:10350000030003271033019300252E00112007F03C
:10351000BFFE084B1B683B40AB4002351E43202DCD
:10352000F4D1019B40C4A342EED1F7BD5CF0004052
:1035300000FEFEFF64F00040802270B5AD4CAE4B43
:10354000D200002120001C6008F042F82300AB4AA2
:1035500088331A60AA4B1A786E23002A00D01133E0
:10356000E3620A232365A74B1878A74BA0630138B1
:10357000E361C3B2032B01D810232362A34B37228C
:103580006361C823DB00A36123008C331A60082326
:1035900036210F3AE518E16323646264E967043970
:1035A000251DE96725003B26BC352E602500C0356A
:1035B0002B602500C4352A6025000636CC352E60E8
:1035C0002500083EC8352E602500D0352960210031
:1035D000D4310B602100D8310A6021000225E0318E
:1035E0000D6025004221DC35296025001B3EE435B5
:1035F0002E602500E8352B602500EC352A6022007E
:103600000525F43215602200F032116022001831D5
:103610009032116022009432136023003C229833D0
:103620001A60AF23DB002360794B2363032805D89E
:1036300007F0EEFE33023537152363609623210031
:10364000FA225B00A360E360C8332361714BFC3155
:103650009200A3640A6062626F4A704DA262732294
:10366000E2656D3A6265A2650232E5644A60022154
:10367000616696218900A166626709210022E166E0
:10368000A2676749674A684E2167E2673560032889
:1036900011D807F0BDFE96089EA61023CDE70E2395
:1036A000CBE70C23C9E720001A259C3005602000D9
:1036B0000735A03005602000A83003602300FA2001
:1036C000F8338000186023006420A43318602300BE
:1036D0005F38AC33186023000338B0331860230020
:1036E000C630B433186023000020B83318602300BC
:1036F0003825FC339D604D4D5A665D644C4D9A648F
:10370000DD619625AD001D624A4D9A675D62F53D0B
:10371000FF3D9D621E25484ADD6618675867D965DA
:103720001966DA67BE23C021444A5B00E250444B6D
:103730004900635004316250C4225200A350FA235E
:10374000E4205B000432A3500432A3503D493E4ABA
:103750003E4BD1603E49800019503E49E938FF3860
:1037600019503D49043019503C491038D1613C4949
:1037700011633C4951633C4911603C49195019009F
:103780003B48F83108603B49D16582213A4A8900BB
:103790005A501A0039490832D1671A003849B432F0
:1037A00011608821374A89005A501A0036498832F8
:1037B0001160364ADA6407F063FF012007F0F8FE73
:1037C00070BD200014259C30056020000435A03019
:1037D00070E7200010259C30056020000335A030E4
:1037E00068E720000E259C30056020000235A030DF
:1037F00060E7C0460004FF1FB865FF1FB070FF1FE1
:103800007845FF1F4A0AFF1F3A07000080C3C9011D
:103810009A02000050C300006A180000280A000045
:10382000204E000088130000F009FF1F0040001127
:1038300068100000C4090000DC05000040420F00D1
:1038400010270000FD1BFF1FFC00FF1F0000FF1FD3
:10385000252FFF1F4D32FF1FE530FF1FD91FFF1F10
:10386000F51FFF1FA121FF1F491FFF1FC528FF1FB5
:103870008D2CFF1FD918FF1FD127FF1F3925FF1FD0
:103880004525FF1F491EFF1F011FFF1FC11DFF1FF1
:10389000F7B50B0CFF270122009300233C001E000C
:1038A0001D009446019089B262469A40100008407B
:1038B00018413618B6B2FF2F02D1012E00D19FB2A7
:1038C000009802401A41AD18ADB2FF2C02D1012D73
:1038D00000D19CB20133102BE6D10320012E07D179
:1038E000012D04D1019B2401E4191C700138FEBD97
:1038F000102EFCD10238102DF9D00230F7E710B5A8
:10390000064C2378002B07D10548FFF7EFFD05484B
:10391000FFF7ECFD0123237010BDC0467865FF1F43
:103920008C65FF1F7C65FF1FF0B58BB00D00012378
:103930000190102936D8FFF7E2FF00231A001B4838
:10394000C15C01335218102BFAD1023B002A29D056
:10395000174B184C1F68002306A9E25C1600FA5C9E
:1039600056405E540133102BF7D102AA07F020FD18
:103970002A0002A9019807F0BBFC07F0E1FC2368CC
:103980001B18236007F0DCFC63681B18636007F0FA
:10399000D7FCA3681B18A36007F0D2FCE3681B18D0
:1039A000E360002318000BB0F0BDC0468C65FF1F1C
:1039B0001844FF1F7C65FF1F0223F0B50124594EF8
:1039C000594D3370594B2C701B688FB0552B10D04C
:1039D000082006F061F900280BD000232100009395
:1039E0000420534A07F014FE8023DB059C62FFF796
:1039F00027FD002006F0E8FB07F002FEFFF79CFD24
:103A000007F07EFD1F22012400214A4B0EAF1A70E1
:103A1000494B1C70494B1970494B19689143163A30
:103A20000A431A60602219689143403A0A431A60B7
:103A300007F04EFD07F08CFDC120FF21414B8000B7
:103A40001A588A431A50C522920098588843BF39A1
:103A50000143995098583C4908408021C9010143CD
:103A6000802099509958C0050902090A01439950CC
:103A700080213648490107F0DBFB0323220034494B
:103A800001940093334807F033FE2C22324903A8F7
:103A900007F03EFE03AC61782078023406F022F98C
:103AA000BC42F8D10121002006F036FA012109209C
:103AB00006F032FA294B2A4A196803201140A02245
:103AC000D2020A431A608022196892040A431A60DB
:103AD0001968244A1140802292030A431A60224B3B
:103AE000224A934200D8012007F0B2FB07F078FB8E
:103AF00007F00EFC307807F0BBFB2878C0B207F067
:103B000077FB07F035FD0A49042007F041FE06F077
:103B100027FB00F09FF800F005FE00F00BFA0020F4
:103B20000FB0F0BD4A0AFF1F7845FF1F34F0004078
:103B30003B000108480AFF1F490AFF1F680AFF1FD0
:103B4000BCF0004000E100E0FF00FFFF7C45FF1FEC
:103B50000058FF1F7C55FF1FA0B7001114F0004054
:103B6000FF7FF8FFFFFF9FFFB070FF1F0080FF1F68
:103B700070B500252849294A29484D6308CA1B0504
:103B80001B0DED188242F9D10022264B8B63264B88
:103B900008211A628022254B9205DA67244BDA68E5
:103BA0008A43DA60234A1278012A03D09A682249AC
:103BB0000A409A600121EE242048E40002686C4328
:103BC0008A430260DA6811208A43DA6007F0B8FAA3
:103BD000112007F065FC112007F082FD184A200C27
:103BE0000400642390420AD8FA220023D2009042B3
:103BF00005D9144B0A21C01807F0B2FCC3B2124A0F
:103C00001372124BD4801B78002B04D1104B10215F
:103C1000187807F09DFA70BD000005408805054042
:103C200000060540FF01000000F0004004E100E054
:103C30003CF000404A0AFF1FFFDFFFFF0038004052
:103C4000B70B000030F8FFFFFC62FF1F3465FF1F59
:103C50002463FF1F002210B51100112007F070FD32
:103C600010BD0000F8B5002301250826394F3A4C55
:103C70003B62E3681120AB43E360E368B343E36076
:103C800007F00EFC112007F05BFA112007F078FC1A
:103C90004023226829001343236080236268DB02EB
:103CA000134380226360A36807201343A360A368C3
:103CB0002A4A1340A3608023A2689B011343102269
:103CC000A360236C93432364236C2B4323648023DE
:103CD0005B003B62226B224B1A402263626B1A40EC
:103CE0006263A26B1A40A263E26B1340E3631D4A56
:103CF000E3681340E36006F0DFF82900072006F0D0
:103D00000BF98021184A1120536C0B43536407F0C0
:103D10002FFDFD21154B164A89005A508023C720DC
:103D2000626B5B0313436363E36880003343E360C8
:103D3000E368104A1D43104BE5601958114080227A
:103D400012020A431A50802292051A600B4B5E63DE
:103D5000F8BDC04600F000403CF00040FFFFDFFF30
:103D6000EFFFEFFFFFFF7FFF003800400000FF1F65
:103D7000713B0011FF00FFFF00E100E00000054083
:103D800030B503A804880B20002C0ED14968074DDC
:103D900008784978090201430A20A94205D1012186
:103DA00020001980024B1B7A137030BD192A0000C5
:103DB000FC62FF1FF7B5150008AA16884A680F4F66
:103DC00014785278120222430A24BA4214D10122F2
:103DD000DBB2019200962A0007F012F9041E0BD103
:103DE000074B1B68002B07D068782A780002104325
:103DF00042425041013098472000FEBD0229000098
:103E00008062FF1F30B5012503790400BFB02B424B
:103E100012D00A49408806F05FFC28420CD06A465E
:103E2000074B69465B8D55801380064B60881B7A73
:103E30001371002203F016FD3FB030BD7862FF1F02
:103E4000C041FF1FFC62FF1F10B50549054806F081
:103E5000F9FB0421044A054806F0B6FB10BDC04634
:103E60007862FF1FFFFF0000CCB70011C041FF1FA9
:103E700010B5024804F078FB10BDC046053E0011A5
:103E80000623837010330371443B43712A338371DB
:103E90004433C37100230222012110B503720E4B7B
:103EA000027041701C8881724472197A0273C17267
:103EB0009A784273DA7882730322C2731A79027491
:103EC0005A7942740C2282749A79C274DB79037530
:103ED0001123C37010BDC046FC62FF1F10B5142033
:103EE00007F0D6FB124B14220021186007F0D8F916
:103EF000002007F025FB012007F0CAFA022007F096
:103F0000CFFB032003F0D4FD042005F0E9FD0520DC
:103F100003F012F8062003F0DFFC072001F06AF836
:103F2000082006F031FB092000F046FE10BDC04617
:103F30008462FF1F10B507F0A3F9012007F0E0FB32
:103F400007F06EFA002010BD094B10B5040098422E
:103F500005D0012904D12000064906F073FB10BDED
:103F60000229FCD1013904F0BDFA0028F3D0F6E7AC
:103F7000FEFF0000AA62FF1F70B50D7A100004AAB0
:103F80002C00168810221440154220D1002E20D17A
:103F90000A78022A18D14A68517815780E4A09021F
:103FA0002943914205D00D4A914209D01C800A2430
:103FB00004E014220A491A8007F09AF9200070BD23
:103FC0000C2208491A80F7E71C800124F6E7082430
:103FD000F4E70B24F2E7C046F3FF0000F4FF000013
:103FE000FC43FF1FACB8001110B504000749084896
:103FF00006F028FB074804F0F7F90020E40704D591
:104000000721054A054806F0DFFA10BDAA62FF1F26
:10401000FFFF0000493F001110B800110442FF1FCC
:1040200000B50C4BBFB01A780B4901A800F0AEFBED
:104030006B4680B25880002809D06A46074B694613
:104040001B881380064B0022188803F00BFC3FB03E
:1040500000BDC0468862FF1F8962FF1F5E42FF1FCE
:104060005E43FF1F00B50C4BBFB01A780B4901A887
:1040700001F03AFB6B4680B25880002809D06A46AE
:10408000074B69465B8D1380064B0022188803F0AE
:10409000E9FB3FB000BDC046B262FF1FB362FF1F25
:1040A0000442FF1F5E43FF1FF7B50E00377A1C0066
:1040B00008AB11003D001A8820231D401F423CD14F
:1040C0003378022B3BD173681F785B781B023B432C
:1040D0001E4FBB4208D01E4FBB4214D01D4DAB42F9
:1040E00021D00A252800FEBD002A2AD1142C2AD866
:1040F0002200F06807F0FCF8174B1C70012CF1D976
:10410000FFF7B0FFEEE7002A1BD1202C1BD82200BE
:10411000F06807F0EDF8114B04211C70104B187873
:1041200007F016F8DEE7E3B20124009201940A00DA
:10413000310006F065FF0500D4E70825D2E7012528
:10414000D0E70B25CEE70D25CCE7C046F3FF0000F6
:10415000F4FF000002290000B262FF1F8862FF1F07
:104160002463FF1F07B5074B01A9188803F066FBFE
:10417000172805D1044B1E224021187807F098F922
:1041800007BDC0465E43FF1F2463FF1F70B51600C6
:1041900004AA148805AA15784A6850781178000294
:1041A0002A4A0843801805284BD807F031F9031331
:1041B0001E29343F0720042C0BD80522121BAA42CB
:1041C00000D92A0022491A803000091907F090F816
:1041D000002070BD0720112CFBD81222121BAA420E
:1041E00000D92A001B491A80EEE707200E2CF0D8D0
:1041F0000F22121BAA4200D92A0017491A80E3E7AE
:104200000720032CE5D80422121BAA4200D92A0059
:1042100012491A80D8E70720032CDAD80422121B8F
:10422000AA4200D92A000E491A80CDE70720032CA4
:10423000CFD80422121BAA4200D92A0009491A80A9
:10424000C2E700220A201A80C3E7C046DCD5FFFF80
:104250005BB80011D062FF1F4BB8001146B80011C7
:1042600041B800113CB8001110B50D21024A0348B5
:1042700006F0AAF910BDC04630B800117442FF1F05
:1042800037B5012000F0BCF81C4D0223002101AA23
:10429000287C00F03BF96A46040002230121287CB7
:1042A000063200F033F9044300F01EF9002C22D14D
:1042B0006B469A882B68D2BA53432A8910491B143B
:1042C0009B184B806B46DA886B6852BA5204520CCA
:1042D00053436A891B0C9B180A481A1C1BB2834261
:1042E00000DD021C130400D500220B888A800133F4
:1042F0000B8020003EBD0124FBE7C046E462FF1FA7
:10430000FC62FF1F0F27000037B5012000F078F88E
:104310001E4D07226946287C00F026F9041E31D183
:104320006B461B787F2B2DD800F0DEF86B46D878D3
:10433000F02302041B031A406B469B8814495BBAA6
:104340009BB21A432B68000953432A891B0C9B1804
:104350004B806B465A789B7812031B011A436B689B
:10436000024353436A891B0C9B181AB21B0402D5E3
:104370008C8020003EBD074B9A4201DC8A80F8E722
:104380008B80F6E700F0B0F80124F2E7E462FF1F4B
:10439000FC62FF1F0F27000010B50E4C237C002B82
:1043A0000CD0382B0BD1012000F02AF8CC22AC2104
:1043B000207C920100F024F900F096F810BD402B0B
:1043C000FCD1012000F01CF80021207C00F0F8F85E
:1043D000F2E7C046E462FF1F10B5084B1A7C002AC2
:1043E00009D05B69002B06D09847041E01D0FEF768
:1043F00007FE200010BD0124F9E7C046E462FF1F5C
:1044000070B500210600162005F0C2FD012115201F
:1044100005F0BEFD07F00CF80400092007F0B0F825
:1044200000222B4B2B4DDA6661321A6019685B3A19
:104430009143002E28D0023A0A431A60AC4209D1B7
:104440000A22DA6107321A6200221A639A63013281
:10445000DA6370BD204A944203D11E22DA6105322C
:10446000F1E71E4A944203D13022DA610632EAE7CC
:104470001B4A944203D14322DA610832E3E7194A26
:104480009442E1D16922F7E702220A431A604622E8
:10449000AC4203D0104A944204D194225A610632AD
:1044A0009A61D1E70D4A944201D1E622F6E70C4A1F
:1044B000944204D13422FF325A610D32F0E7094AA6
:1044C0009442C1D1E62252005A610A32E8E7C0465E
:1044D000005000400024F4000048E801006CDC02B9
:1044E0000090D00300D8B80510B50024064B092071
:1044F000DC6606F0D5FF2100162005F0DDFC21006A
:10450000152005F0D9FC10BD00500040F8B51C0086
:104510000023134D0F00EB666860160006F038FEAE
:1045200001238022EB6623002F615200013B08D259
:1045300006F016FF08200B4A1168002C03D120005A
:10454000F8BD2A61F2E72B6F034203D02B69013CCF
:104550003370013613685B1A012BEED90124EEE7A4
:10456000005000406008FF1F002370B5124D14007A
:10457000EB6668600E0006F00BFE01238022EB66FE
:1045800023005200013B08D206F0EAFE08200B4A45
:104590001168002C03D1200070BD2A61F2E72B6F57
:1045A000034203D02B69013C3370013613685B1A58
:1045B000012BEED90124EEE7005000406008FF1FF8
:1045C000002370B50C4C0D00E366606006F0E0FD62
:1045D0000123E366256106F0C3FE8020074A8000C0
:1045E0001168636B034205D113685B1A012BF8D97C
:1045F000012070BD0020FCE7005000406008FF1F54
:10460000002370B5134C0E00E3666060150006F0E1
:10461000BFFD0123E36626610F33626B1A42FCD0B3
:104620002B0A23611023626B1A42FCD0EDB2256184
:1046300006F096FE8020084A80001168636B0342F2
:1046400005D113685B1A012BF8D9012070BD002039
:10465000FCE7C046005000406008FF1F0A4B0B4AB1
:1046600019689068884202D980235B04C91853688E
:1046700091601B1A5B181168D80B5B0440185B0C27
:10468000106053607047C04628F000401463FF1F5D
:1046900010B51B4B1A793F2A01D93F221A7119799B
:1046A000184A1948117018221849028018480A80BF
:1046B00002804A809A791748802402800C208A80E0
:1046C000013242432401101CA24200D9201C124A8C
:1046D000C88010805A79002A01D101325A711A7AA1
:1046E000012A01D802221A725A791B7A0B485343C5
:1046F0000A21584306F034FF094C206010BDC04623
:104700000863FF1F480AFF1F5C43FF1F2445FF1F6C
:104710005A43FF1F0065FF1F5843FF1F710200002F
:104720002863FF1F10B507210020FEF751FE124C31
:10473000002807D10C222000104906F0D9FDFFF710
:10474000A7FF10BD0C2220000D49FEF715FE0C2816
:1047500004D00C222000094906F0CAFD094C0C22A5
:1047600020000949FEF708FE0C28E8D00C220021A1
:10477000200006F095FDE2E70863FF1FA0B80011D6
:10478000FC0C0000E462FF1FF50C0000F0B5040013
:104790000D00160085B0002A00D1C8E0087800217D
:1047A00020706170262800D18EE00FD8072805D828
:1047B00006F02EFE502B2B2B2B95A39C232800D1EB
:1047C000B7E0252868D0FF236370A5E0712800D1E9
:1047D0009AE014D8552845D05628F4D1854D0C229E
:1047E0008549280006F084FDFFF752FF0C2283491B
:1047F0002800FEF7FBFC0C222900601C46E0722812
:1048000000D18BE0DC2800D1ABE0DB2800D0C5E094
:10481000042ED8D9AA786B7812021A43EB781027A5
:104820001B0413432A7912061A430192052E05D060
:10483000771F3A000198691D06F05AFD05222900EC
:10484000200006F055FD3A000199601D06F050FD6C
:10485000781D05E00C222000694906F049FD0C2076
:1048600005B0F0BD013A634E0C2A13D8002A0AD0D5
:10487000691C300006F03CFDFFF70AFF0C223000F7
:104880005E49FEF7B3FC0C223100601C06F030FDDF
:104890000D20E5E70C22EBE7013A5A4E0C2A11D81D
:1048A000002A08D0691C300006F022FD0C223000DE
:1048B0005549FEF79BFC13223100601C06F018FDE1
:1048C0001420CDE70C22EDE74E4D1322280006F010
:1048D000E7FCFEF795FB13222900601CEEE705229A
:1048E0004A49601C06F004FD0620B9E71222484937
:1048F000601C06F0FDFC1320B2E708224549601C4D
:1049000006F0F6FC0920ABE76978F72900D95AE7E9
:10491000414B188801F048FB0220A1E700F056FB4C
:10492000012E02D06A783D4B1A6006F0F9FB002098
:1049300096E7013A3A4E042A11D8002A06D03000F0
:10494000691C06F0E5FE374B1B68B360FFF786FE77
:1049500004223100601C06F0CBFC052080E7042215
:10496000EDE7022A00D82EE76B786370AB78A3706E
:104970006F781B021F43032A05D0033E3900B2B2F1
:10498000E81CFEF733FC10223900E01CFEF7F4FCB3
:1049900003000330002B00DB62E715E7DA2800D0C4
:1049A00011E7042E00D80EE7AB786A781B02134398
:1049B000EA7812041A432B791B061343082E16D9E2
:1049C000AA79697912020A43E979090411432A7A1A
:1049D00012060A4303921A601B6805222900200070
:1049E000039306F085FC0422601D03A988E7FE22DC
:1049F0006270F1E70863FF1FA0B80011FC0C000013
:104A0000ACB80011E462FF1FF50C0000F062FF1F5C
:104A1000D062FF1F9844FF1F5E43FF1F34F0004029
:104A20001463FF1F28F0004070470000013870B584
:104A3000042809D806F0ECFC030920081200184BE2
:104A40000221187806F084FB70BD154B08211878F8
:104A500006F0C6FD0022134B1A72F5E70024114B35
:104A60000F4D082128781A681C8106F0E1FD21000D
:104A7000287806F055FCE7E7094B0821187806F07E
:104A8000AFFD0948FFF7FCF9084B094A9B79938071
:104A9000084A13808022034B52001A81D4E7C04693
:104AA0002463FF1F2863FF1F6743FF1F0863FF1F67
:104AB0002445FF1F0065FF1F10B5002903D1092001
:104AC000013105F029FA10BD020010B5094B0A3278
:104AD000094C92B2DA815A8298811882207802F0C9
:104AE000C9F80422054B012120781A7006F030FB2A
:104AF00010BDC0462244FF1F6265FF1F6165FF1F96
:104B000010B501290DD10021092005F005FA054B4A
:104B10001B78002B05D02622034B04485A72FFF75E
:104B2000D3FF10BD3465FF1F2863FF1FC4090000B9
:104B30000300F0B50A4D8E18B14202D15200801820
:104B4000F0BD0C782F6824093C5D0F271C700C7891
:104B500001313C402F683C5D5C700233ECE7C0469D
:104B60005443FF1F10B5114B1A781870002A0ED04D
:104B700000280BD10E4B1A78062A07D85423D340AD
:104B8000DB0703D50B4B187802F074F810BD002832
:104B9000FCD0074B1B78012B02D0033B022BF5D82E
:104BA000044B0121187806F0D3FAEFE73465FF1FB4
:104BB0006165FF1F6265FF1FF7B5604D604A61497F
:104BC0002870082005F0AAFA0121092005F0A4F9AF
:104BD000092005F08DFA0121002005F09DF9002043
:104BE00005F086FAFEF70CFA06F012FB032256498E
:104BF0005648FFF79DFF2D24030004221C705449E2
:104C00000130FFF795FF3023022204704370837058
:104C1000504C514B2000DA8706F0D2FB022815D009
:104C2000062220004D49FEF7A7FB06280ED00321DF
:104C3000200006F09DFB8D23E3706E3B237106225E
:104C40001933200045496371FEF7D0FA0E23444F13
:104C5000444C454E3B70013B0522300043492370D4
:104C6000043B6370019606F043FB2D23012240496B
:104C70004048E371FFF75CFF01223F49FFF758FF0F
:104C800001223449FFF754FF0020FFF76BFF3B4E32
:104C90003B4A01213B4B1278307801F0ADFF2300F5
:104CA00000213A78307801F0A7FF01222178364BB5
:104CB00001391A700020019AC9B205F0A3FB334BE9
:104CC0001A68552A30D100221A60314B3C323148E3
:104CD0005A72FFF7F9FE2021287806F009FC01201E
:104CE000404205F0DBFB0120404205F077FCFFF776
:104CF000BBFAFFF7A9F800F08FFC01204042FFF754
:104D000073F9012006F09CFCF72001F031F9012134
:104D1000287806F01DFA287802F008F91E4806F0F7
:104D20003FFBFEF79FFFF7BDFA210B4B1B4A4901E2
:104D30009981DA8119825A82CDE7C0462463FF1F28
:104D4000B94A0011014B00119844FF1FD062FF1FA8
:104D5000F062FF1F6509FF1F2244FF1FADAC00007A
:104D60003065FF1F1165FF1F1365FF1F5BB8001142
:104D70006709FF1F1965FF1F6609FF1F6265FF1F97
:104D80008643FF1F6743FF1F0265FF1F34F000408B
:104D90002863FF1FC40900003463FF1F4A1F00007F
:104DA000F8B50A0020230D001A40194239D0474BAC
:104DB0001B78002B23D0FFF751FC454C454E636810
:104DC000727AC31A934202D36060FEF74BFF327AC5
:104DD000217A531EDBB2994214D1FFF7DDFA637AD0
:104DE000002B09D0013BDBB26372002B04D1707938
:104DF00064335843FFF768FE237A0133237220207F
:104E00006840F8BD9142EAD300232372FFF7E4FA29
:104E1000314F3800FFF734F83900152006F0E8FB71
:104E2000DDE70BB2002B0ADA2C4B187806F068FA93
:104E3000002801D006F0CCFA80200002E0E702242E
:104E4000214206D0224B01201A72FFF78BFE200070
:104E5000D6E70B0713D5FFF701FC1D4A1D49536820
:104E6000497AC31A8B4202D35060FEF7FBFEFFF76C
:104E7000B3FAFFF791FA00F0E9FB0820C0E710242D
:104E80000E002640214206D0104B1B78002BDED1AD
:104E9000FEF7EEFFDBE70124214209D0104800F0C5
:104EA0006DF806F00DFA3100092005F035F8CEE76F
:104EB0004024214202D0FFF755F9C8E70424080036
:104EC000204021429DD0FFF7ABF8C0E73465FF1FBB
:104ED0002863FF1F0863FF1F6743FF1F2463FF1F33
:104EE0004C43FF1FF0B51B4B1B4F1B883A88040037
:104EF0001A4E1B4D85B09A420DD832889A420AD379
:104F0000184B1A882B889A4205D1174A174B1288DA
:104F10001B889A421BD0052001F080F83B8802AA2A
:104F200013803388019053802B88114D93800F4B51
:104F300002A91B88D3800F4B2A78188802F09CFDA9
:104F40000D4B08212878019A1C7006F0B1FA05B0C3
:104F5000F0BDC046FE64FF1F5C43FF1F5A43FF1FA6
:104F60000065FF1FFC64FF1FFA64FF1F5843FF1F0B
:104F70006265FF1F5E43FF1FF864FF1F13B50C4BF4
:104F80001C78002C11D1002801D00A4B18600A4A65
:104F90000A4B11780A4A10780A4A01920A4A00928A
:104FA000002205F027F9200016BD1124FBE7C046BA
:104FB0006165FF1FF464FF1F6065FF1F5065FF1FE1
:104FC0006265FF1F3C65FF1F4065FF1F10B5064B64
:104FD00012201B78052B06D1044B13221988044B91
:104FE000187801F0F7F910BD6165FF1F5E43FF1FE0
:104FF0006265FF1F10B500240122114B5242187048
:10500000104B1C70104B1A8001F090FF04220F4BC4
:1050100021001A700E480C3206F042F910222100CD
:105020000C4806F03DF907220B4B1C600B4B1C7023
:105030000B4B1C700B4B1A700B4B1C7010BDC046F9
:105040006265FF1F6165FF1F5E43FF1F6065FF1FF5
:105050005065FF1F4065FF1F3C65FF1F1065FF1F68
:105060000F65FF1F6043FF1F0E65FF1FF8B5174C4C
:105070000600257806A814240078052D23D1B41F36
:10508000134FA5B21824BD421DD88D1FADB2BD422D
:1050900019D8FA256D00AA4215D21D000D4F0A3D00
:1050A000ADB2BD420FD80C4C26800C4C21800C496F
:1050B00000240A800B4A1380FFF714FF0A4B0421D7
:1050C000187806F08DFA2000F8BDC0466165FF1F14
:1050D000790C0000750C00005C43FF1F5A43FF1F52
:1050E0000065FF1F5843FF1F6265FF1FF0B50BB23D
:1050F0000D0089B0002B00DB76E1A64E307806F07B
:10510000FFF8041E55D00378A22B00D127E1D02B45
:105110001AD0912B4AD143780E2B47D19E4B8288CF
:105120009A4243D19D4A83681278052A3ED10320D2
:1051300018567F283AD09A4B1B68002B36D05B68F4
:10514000002B33D0984731E0807807282ED806F01E
:105150005FF9042D1D444479ADDD6378002B11D136
:105160000622E11C8F4806F0C3F801218B4B197011
:105170008D4B1A78002A5BD08C4B307801F03CFDC7
:10518000002855D00722854B1A7051E0617800291C
:10519000F8D1E378002B11D0854A864B127830780D
:1051A00001F02AFD60706378002BEBD1200006F03F
:1051B0000FF980200002684009B0F0BD774B1B78E2
:1051C000022BF3D00121307806F02AF80028EAD12A
:1051D0000121307805F0BCFFE5E76378002BD1D1E1
:1051E0006E4F032807D13B78052B02D101333B706A
:1051F0001EE00223FBE7704B1A88704B0293002AD3
:105200000BD01B78002B03D00121307806F050F929
:105210003B78062B04D1013BE9E7029B1A70F7E7C4
:10522000042B41D10121029B3078197005F090FFC9
:105230005B4B1B68002BB9D01B68002BB6D0574ABC
:1052400010787FE76378554F002B27D10622211D68
:105250005B4806F04DF862895A4B5B491A80A28977
:105260005A4B1A80E3890B800521397058490A800E
:10527000584A1380228A584B1A80584B1B78012BAE
:1052800009D11F2000F0CAFEFA22920042430421F5
:10529000307806F00DF90022484B75E7312B00D02D
:1052A00070E70022454B1A700323A0E70622002175
:1052B000434805F0F5FF0023454A04211380454A81
:1052C00030781380444A138006F08AF90821307838
:1052D00006F086F9A379083B5A4253412F4A03331B
:1052E0001370314B1B78002B06D0344B30781A7872
:1052F000002A06D001F0BEFC0122324B52421A8035
:1053000096E70121197005F023FFF5E708213078B1
:1053100006F066F96378002B00D047E72C4B2E4F40
:105320000293E388029A042113802A4B3078039376
:105330002389039A138063893B8005F071FF00285D
:1053400000D033E7264B1B68002B00D12EE70399D2
:1053500002983A88098800881B68984726E74379AD
:10536000132B00D022E70389012B0AD11D4B1B7898
:10537000022B06D10821307806F032F9FFF726FE1D
:1053800014E7052000F04AFE08210200307806F0FC
:105390008FF80BE76265FF1F051400006165FF1FB2
:1053A000F464FF1F3565FF1F8643FF1F6743FF1F20
:1053B0003065FF1F1165FF1F3265FF1F3465FF1F3A
:1053C0000365FF1F5E43FF1F0A65FF1F0C65FF1F7C
:1053D000FE64FF1FFC64FF1FFA64FF1F0265FF1FCE
:1053E000F064FF1FF864FF1F8020C001014200D05D
:1053F000E1E6CB0731D5324B1B78002B1DD0314E67
:1054000005AC3378052B1AD1023B23702E4B2100BB
:105410001B7823722D4B1B7863722D4B187801F08B
:105420008FFB002809D007202A4B30701B68002B07
:1054300003D01B68002B00D098470120BBE60E204C
:10544000254B06221B7825492370254B1B7863705A
:1054500002ABC01805F04CFFD8E702230800184043
:10546000194209D0174B1B78052B03D11D4B188807
:1054700006F006F802209EE60424214203D0FFF73E
:1054800031FD200097E6082308001840194200D19A
:1054900092E6154B1C78012C03D0022C0DD008206D
:1054A00089E6124B124A134913481B88128809884F
:1054B00000880094FFF7DAFDF1E7FFF787FDEEE7DC
:1054C0003465FF1F6165FF1F6043FF1F0E65FF1FEF
:1054D0006265FF1FF464FF1F1065FF1F6143FF1F1C
:1054E0000F65FF1F5E43FF1FF864FF1F5843FF1F38
:1054F0000065FF1F5A43FF1F5C43FF1F10B502A842
:1055000004880B20002C10D14968087849780902DA
:1055100001430C48814209D1022119800A4B598864
:105520001170DB7800205BB2537010BD074C0A206D
:10553000A142FAD102211980034B998811705B793D
:10554000F0E7C0466E2A0000FC62FF1F6F2A0000D1
:10555000F7B5150008AA16884A680F4F14785278D4
:10556000120222430A24BA4214D10122DBB2019270
:1055700000962A0005F044FD041E0BD1074B1B6862
:10558000002B07D068782A7800021043424250412D
:10559000013098472000FEBD022900007465FF1FFE
:1055A00030B5012503790400BFB02B4227D015493F
:1055B000408805F091F828420DD06A46124B6946A2
:1055C0005B8D138002235380104B5B88938060882F
:1055D000002202F047F90E49608805F07DF8C00707
:1055E0000DD56A460B4B69461B88138002235380F6
:1055F000064B9B8893806088002202F033F93FB00D
:1056000030BDC0466C65FF1F8843FF1FFC62FF1F53
:105610006465FF1FE243FF1F10B5074C07492000D8
:1056200005F010F82000064905F00CF80721054A9E
:10563000054804F0C9FF10BDFFFF00006C65FF1FA7
:105640006465FF1F2CB900118843FF1F10B5024885
:1056500002F08AFF10BDC046A15500110200F0B54E
:1056600001270A480A4E51188B1A002B00DCF0BDA6
:10567000082415784308684038404000805B013CAE
:1056800058406D08002CF5D10132EDE7FFFF000016
:1056900046B90011F0B500250F269D4200DBF0BD94
:1056A0004C5D070944403440A400A05801357840BF
:1056B000F3E70000F0B589B06A460D000B000F2734
:1056C000110010351C780133260024093E40167065
:1056D00054700232AB42F5D12023024AFFF7DAFFC1
:1056E00009B0F0BD4CB90011F0B54E780B7889B017
:1056F00036020C00170001901E43012A61D9974B16
:105700009E4200D877E001339E421CD1062A17D171
:10571000CA788B7812021A430B791B0413434A7917
:1057200012061A438E4B5A6100221A705A808D4A13
:105730005A608D4A9A608D4ADA60002009B0F0BD47
:1057400088225205EEE78A4B9E423CD184498B78F1
:10575000002B00D0F9E00C2A31D10F22A37893431B
:10576000E27812021343227912041343627912067B
:1057700013434B60E279A07912020243207A0004BD
:105780001043627A12060243CA60E27AA07A1202D9
:10579000024378484A81834208D80423704914227E
:1057A00001980B7005F0A4FD1420C7E71201D21870
:1057B00089235B059A42F0D801238B70BDE7022A4A
:1057C000FAD00523EAE76C4A01239642E6D1FFF7B7
:1057D000FDFB052F0CD9E378A2781B021343227935
:1057E00012041A4363791B061343644A039313603C
:1057F00005F096FCA1E75A4D2B78002B9DD1AB7894
:10580000002B00D1A3E02B8901339BB20093B3425C
:1058100000D094E0132AD4D9CF7C8B7C3F02122194
:1058200020001F43FFF71AFF874200D091E0002EAF
:105830003ED1E378A2781B0213432279E96812046F
:105840001A4363791B06134303930A228B4213D135
:10585000FF23A370E370237163716B89002B0AD15E
:10586000E37B227C1B0212041343A27B13430393AA
:105870001B0901336B8100226B89002B8DD0002A1C
:1058800069D1686837013818000B6B690003039011
:10589000984205D9686105F09BFCEB780133EB7009
:1058A00068681022A11C381805F09AFD2E8144E783
:1058B0006F89009A7B1E9BB293423CD1E378A27819
:1058C0001B02134322792E4E12041A4363796C682B
:1058D0001B0613433100042204A8039305F008FDBE
:1058E000211D0C2205A805F003FD012004A940425A
:1058F0001034FFF7DFFE013F012F17D1039A0B236E
:105900002861824200D049E704223100686805F02E
:1059100067FD042203A9686805F0D2FEE968039ACE
:10592000FF23914200D139E7F73B37E72100FFF72A
:10593000C1FE1034DFE70923B742A2D82EE7009B4F
:10594000B34200D9F9E6072328E7022326E7032319
:1059500024E7062322E70A2320E7C046FFFE0000D3
:10596000FC43FF1F00000111FFFF000050485936A3
:1059700001FF0000FFFF001102FF000034F00040B3
:105980000844FF1F10B5034C0B000122210000F05A
:105990006BFA10BD455B00110B8870B506000D0059
:1059A0000224162B11D92B000322094900F05CFABE
:1059B000041E0AD1074B2A881B88191C934200D960
:1059C000111C300089B200F0EFFA200070BDC04613
:1059D000715B0011D265FF1F10B54A780400013ACF
:1059E0000B000220012A07D80A78002A04D00522D9
:1059F0002000024900F038FA10BDC0469F5B00113C
:105A00000A7810B50B0004000220002A04D00722F7
:105A10002000024900F028FA10BDC0464B5C00117E
:105A20000A7810B50B0004000220002A04D00922D5
:105A30002000024900F018FA10BDC046B15C001108
:105A400010B5034C0B000B22210000F00DFA10BD25
:105A5000E15C001110B5034C0B000D22210000F099
:105A600003FA10BD535D001110B5034C0B000F225B
:105A7000210000F0F9F910BDAD5D00110A7810B5F4
:105A80000B0004000220002A04D011222000024949
:105A900000F0EAF910BDC046BD5D0011002310B54D
:105AA0001322190000F0E0F910BD000010B5034CFE
:105AB0000B001722210000F0D7F910BD0F5E001176
:105AC000002310B51922190000F0CEF910BD000016
:105AD00010B5034C0B001B22210000F0C5F910BDCE
:105AE000495E0011F7B584890D0006000121002CE4
:105AF00022D000238268D3561778002B1EDA0C2C94
:105B00001AD90C3CA4B2131940880093230002F068
:105B100086FE431E984101307B06DB0F6B703F23EE
:105B2000013C1F40A4B22870AF70AC80002C07D09D
:105B3000B3680133AB6000210800FEBD0020EBE735
:105B4000AC60F8E70B7803704B8843704B881B0AF6
:105B500083700B79C370042070470420022B06D198
:105B60000020537811781B02009A0B431380704772
:105B70000B8803700B881B0A4370022070470420B7
:105B8000009983420AD1537810781B0203430B809B
:105B9000D37890781B02034300204B807047F8B500
:105BA0000D004B7801240021461C03702B788B429A
:105BB00001D82000F8BD6B78B01C4F1C012B10D110
:105BC000890069184B88022233704B88B9001B0A80
:105BD0007370691805F08CFB04360434A4B2F9B272
:105BE000E4E7122359436B185A88043132705B88FA
:105BF00010221B0A7370691805F07AFB12361234F2
:105C0000ECE770B5049D14001E00052B01D804209C
:105C100070BD637812781B0213432B80E378A2785F
:105C20001B02134302226B802A71211D681D063E50
:105C300005F05EFBB2B22A81F02AE8D82800A11D47
:105C40000A3005F055FB0020E2E7002310B50A7882
:105C50009A4201D8900010BD9A008A1854880133E6
:105C600004705488DBB2240A44709488847092884B
:105C7000120AC2700430EAE710B51100029C062B2C
:105C800004D004201022142B01D010BD0222227156
:105C90004B7808781B0203432380CB7888781B025B
:105CA000034363800431601D05F022FB0020ECE714
:105CB00010B50C788B7804315C43E4B20370220099
:105CC000013005F015FB601C10BD0420022B06D12D
:105CD0000020537811781B02009A0B431380704701
:105CE00010B50C000A88023105F002FB208810BDB7
:105CF00070B504000D0004981100012B01D8042098
:105D000070BD167852781202324302800200F832D7
:105D100055701470E825002C00D10C35023B9AB266
:105D20004280AA42EBD80231043005F0E1FA0020AB
:105D3000E6E70420009983420AD1537810781B02C9
:105D400003430B80D37890781B02034300204B80E1
:105D5000704710B50C000A88023105F0C9FA208896
:105D600010BD000070B501211E000420049C0E40EF
:105D70000B4218D1CB40DDB28D4214D90A49DBB2B7
:105D8000098899420FD32300F6331D703300580061
:105D900011184978165C0902314301332152D9B2F6
:105DA0008D42F4D8002070BD1C44FF1F10B50C00BC
:105DB0000A88023105F09CFA208810BD10B50C78D5
:105DC0008B7804315C43E4B203702200013005F0AB
:105DD0008FFA601C10BD10B511000298032B01D87A
:105DE000042010BD14785278043B12022243028032
:105DF000CA788C781202224342809AB28280F22AB8
:105E0000EED80431063005F073FA0020E9E710B54A
:105E10000C000B8803700B881B0A43704B8883703F
:105E20004B881B0AC3708A880430063105F060FA7B
:105E3000A088043080B210BD0420012B03D10020C3
:105E40001378009A1370704710B50C000B8803701C
:105E50000B881B0A43704A880230043105F048FA67
:105E60006088023080B210BDF0B589B003931E4B3C
:105E7000029242000700D05A019102F020F8132547
:105E8000061E2DD0029B01240370019B002B04D021
:105E9000001903999847001984B26B461B7A5BB2CC
:105EA000002B0FDA1021380002F01CFB1925002806
:105EB00013D130003219E1B202F066FC051E0CD19C
:105EC0000C34A4B2042304AA380005A993800696D2
:105ED000948101F0AFFD051E02D0300005F028FAD4
:105EE000280009B0F0BDC046D065FF1F70B50500A1
:105EF0000C0000280CD00020814209D01022200084
:105F0000044905F0F5F901202B7823736B7863734E
:105F100070BDC0468CB90011F0B506000D00170029
:105F20001C0085B002291BD00020102907D1022BAC
:105F300007D0102B03D115E00020102C08D005B09D
:105F4000F0BD69463800FFF7D1FF2A0069460BE033
:105F500069463000FFF7CAFF22006946380004E0B6
:105F6000022BE9D12A003900300005F081FAE6E77A
:105F7000031CF72800D9F723032008499AB2013AF5
:105F80000B80D317034006499B189B100B80D30F3F
:105F900004499B185B100B807047C0462044FF1FCC
:105FA0001E44FF1F1C44FF1F034B1B888B4202D360
:105FB000024B4000C15270472044FF1FD065FF1FB5
:105FC000014B4000185A7047D065FF1F1722014B44
:105FD0001A807047D065FF1F70B505000E2005F0D0
:105FE000DFF8041E13D0D023037000230622837031
:105FF00007494570033005F07BF9064B2100DA8A2A
:1060000062811B7E2373044B187805F0A9FB70BDD9
:10601000EC65FF1FDC65FF1F7044FF1F262803D8B7
:10602000024B4000C05A70470148FCE72244FF1F62
:10603000FFFF000070B506000C00094D1C22002176
:10604000280005F02DF9074B1E70074B1C7005F05A
:106050006FFB0123002801D0002312202B7070BD9C
:10606000DC65FF1F7044FF1FFD65FF1F70B5050055
:106070000D4C0800E260A16010220021656005F06F
:10608000BFF9012803D11021A06802F058FD1022A9
:106090000021280005F0B4F9012803D1102160681F
:1060A00002F04DFD70BDC046DC65FF1F70B5041EDB
:1060B00005D1002903D006220D4805F019F90D4B32
:1060C0001D78012D11D1002C05D102221A7005F086
:1060D00067FA280070BD00221A70074B1B78FF2B4F
:1060E000F7D02000FFF778FFF3E70025F1E7C0467F
:1060F000EC65FF1FDC65FF1F7044FF1F030010B538
:10610000002801D1002010BD00780B4A002803D1DF
:106110005988D1821B7913761378022BF2D1002390
:10612000984200D103331370044B1B78FF2B01D02E
:10613000FFF752FF0120E6E7DC65FF1F7044FF1FF9
:10614000002911D000280CD04B79012803D140221E
:106150005242134303E03F221340032802D00120A0
:106160004B7170474022F4E70800FAE770B5094D1B
:106170000100287800280BD0074C0622200005F0EB
:10618000B7F821002878FFF7DBFF200005F098F929
:1061900070BDC046FC65FF1FD665FF1F00290AD0F1
:1061A000012808D13F224B799343C02B03D0403BB9
:1061B0005A425341981C704770B5174D06002B7812
:1061C000FF2B15D00A2004F0EBFF041E10D0D023C3
:1061D0000370C83B8370114B11491B784670C37024
:1061E0000622043005F084F82100287805F0B8FA7A
:1061F0000C4B1B78012B0DD10B4B1B68002B03D0D4
:106200009B68002B00D09847084B04211878084A57
:1062100005F00EFA70BDC0467044FF1FFC65FF1FFD
:10622000D665FF1FF865FF1F2466FF1F2866FF1F46
:1062300060EA0000014B98687047C046DC65FF1FAC
:10624000014BDB6818687047DC65FF1F074B10B512
:10625000DA68136801331360054B1878FF2803D000
:106260008021C90104F074FF10BDC046DC65FF1F2A
:106270007044FF1FF7B50E0002F0C8F8051E1CD0D1
:106280000E4B06621F78002F00D10778AB791020E3
:10629000019304F085FF041E0FD0D0230380C73B79
:1062A0008370019BE91DC3700622043005F020F8BD
:1062B00021003800E66005F053FAF7BD6E44FF1F79
:1062C000014B18787047C046FC65FF1F054B00283E
:1062D00005D1054B1A78054B002A00D1014B180057
:1062E0007047C046EC65FF1FFC65FF1FD665FF1FAA
:1062F000014B58687047C046DC65FF1F024B1868A9
:10630000431E9841C0B270470066FF1F421E030043
:106310000120152A03D9FF3B5A425341D8B2704796
:10632000F0B51C0000230E0085B0039002920B70A4
:10633000029A934201D3002019E0E55C5A1CD2B2C4
:10634000002DF8D0029851198142F4DC0233DFB2FB
:10635000A35C18000193FFF7D9FF002807D0013D87
:10636000019A0399EBB233708A4202D1E01905B069
:10637000F0BDDB19DBB2DBE710B50C0002F09EF8D4
:1063800003001220002B03D02100588805F068F884
:1063900010BD000070B50E4D84006359002B15D060
:1063A000186A002801D005F023F82B59586A0028F4
:1063B00001D005F01DF82B59986A002801D005F08E
:1063C00017F8285905F014F800232B5170BDC0466A
:1063D0000C66FF1F1C4B70B504000E00150099429F
:1063E0000AD11A4B1B68002B01D1122070BD1B680B
:1063F000002BFAD09847F9E7154B994215D1134B6A
:106400001B68002B0AD01B68002B07D09847002878
:1064100004D1104B1C70104B1D70E7E729002000C1
:10642000FFF7AAFF0028E1D1F3E7080001F0EEFF33
:106430000028DAD003780320A342D7D12900300006
:1064400005F00EF8D2E7C046FEFF00000866FF1F09
:10645000FFFF00000566FF1F0466FF1FF7B504007D
:10646000808801F0D3FF0025A84203D00578A088DA
:1064700002F008F81C4E3378002B1FD0AB421DD120
:106480001A4B28001978FFF777FF002818D000234F
:106490003370A3790820A778A688019304F080FEC2
:1064A000011E0DD0D0230370CA3B8370019B47703F
:1064B00086808371280005F053F901E0002DE8D1B2
:1064C000A0880B4B8200D358002B01D0FFF762FF4E
:1064D0001721A088FFF768FDA08801F027FDA0889C
:1064E00001F0FEFDF7BDC0460566FF1F0466FF1FF5
:1064F0000C66FF1FF0B587B01D000CAB1B880700B2
:1065000001930DAB1B88142002930EAB1B88160061
:1065100003930FAB1B880091049310AB1B8805936A
:1065200004F03EFE041E1AD0D0230370CB3B47700C
:106530008370C670062229000430002D11D004F0AB
:10654000D7FE019B21006381029B0098A381039BDE
:10655000E381049B2382059BA37405F001F907B036
:10656000F0BD04F09DFEECE7F7B5009308AB1B8887
:1065700007000C200D001600019304F011FE041E0C
:1065800013D0280001F042FF00280FD00078D0235C
:106590002370C93BA370009B21002381019B67707E
:1065A000A580E680638105F0DBF8F7BD014B187824
:1065B000EDE7C0467044FF1F13B5040064890389EA
:1065C000C2888188C0780094FFF7CEFF13BD000019
:1065D00010B5044C2068002803D004F009FF002304
:1065E000236010BD1066FF1FA122F0B581889200C4
:1065F0004A43384B384F1B6804009B189D22920079
:106600009B18827989B01A603B68002B5FD01D7897
:10661000324B1B68002B04D05B68002B01D000209C
:106620009847260008363100E079FFF7B7FD237D53
:10663000E0710200E0780493638A29000393238ABF
:106640000293E3890193A38800933300FFF752FF7D
:10665000E378002B0BD1E289A379A18802920196FD
:10666000E27928000092012201F0DAFEE0703B6836
:10667000002B20D0FFF7ACFF194D287800281AD046
:10668000184B1978FFF778FE002814D02B78E6789D
:1066900008200793A78804F083FD011E09D0D023AA
:1066A0000370CA3B4670837087808671079805F037
:1066B00057F800232B701721A088FFF775FCA088DE
:1066C00001F034FCA08801F00BFD09B0F0BD064BD1
:1066D0009DE7C0463409FF1F1066FF1F2466FF1F99
:1066E0000566FF1F0466FF1F7044FF1FF8B5070013
:1066F00008000E0001F08AFE041E18D02620FFF7C5
:106700008DFC051E00D12578062004F049FD041EED
:106710000DD00021062204F0C3FDD0232370C23B1C
:1067200021006770A370A680E8B205F019F8F8BDE3
:10673000F0B585B001930AAB1B78070002930BAB51
:106740001B7808000D000092039301F05FFE061E07
:1067500022D0102004F024FD041E1DD010220021A0
:1067600004F09EFD2620FFF759FC002800D1307868
:10677000D0232370C13BA370009B21002372019B97
:1067800067706372029BA580A372039BC0B2E37221
:106790000C9BE36004F0E4FF05B0F0BDF7B50D001D
:1067A000019001F033FE071E20D00E2004F0F8FC0B
:1067B000041E1BD02620FFF731FC061E00D13E78B8
:1067C000D0232380C53B0622A370F91DE01C04F0F2
:1067D0008FFD019B2A0063810123DD401A401D408B
:1067E000210022736573F0B204F0BAFFF7BD000018
:1067F000F0B585B0029010000D0017000A9E0393BB
:1068000001F004FE041E31D0029B002B2ED1039B0D
:1068100002795B0724D5122313430422002E08D1EA
:106820000B99002905D10C99002902D10D99002955
:106830001AD01A430D9B2271002B00D0C9E0002E04
:1068400000D1CFE0002D00D0CCE0606A002801D05C
:1068500004F0CEFD1C21300004F06AFC606205E00B
:1068600002239A430E33D7E793432371654BBA0053
:10687000D458002C00D1AAE0002E10D0236A002B9F
:1068800003D11C2004F004FF20625E4BBA00D358F1
:10689000186A002803D01C22310004F029FD0C9B4B
:1068A000002B12D0574CBB001D596B6A002B03D133
:1068B000162004F0EDFE6862BB00E358586A002819
:1068C00003D016220C9904F013FD0D9B002B11D060
:1068D0004C4DBC006659B36A002B03D1142004F060
:1068E000D7FEB0622B59986A002803D014220D9964
:1068F00004F0FEFC380001F089FD051E67D0414B15
:10690000BA00D358002B62D01A6A3420002A00D172
:106910001C389A6A002A01D0143080B20B9A002ADF
:1069200001D01C3080B25B6A002B01D0163080B2DF
:1069300004F036FC041E4AD01822002104F0B0FCFA
:106940002620FFF76BFB0190002801D12B780193E3
:10695000D0232370029B200063700A23294EA3706A
:10696000039BBD00A371AB59A780196A1830002999
:1069700005D01C22A06004F0BBFC20003430735909
:10698000996A002907D0030014221433E0600293AF
:1069900004F0AEFC02980B9B002B08D003001C22D5
:1069A0001C330B992061029304F0A2FC02987359E6
:1069B000596A002903D01622606104F099FC6B46E5
:1069C0002100187904F0CCFE3800FFF7E3FC05B095
:1069D000F0BD10220D9B0D991B69A018236204F0D5
:1069E00087FC2CE70B9B002B00D13FE7012D00D04B
:1069F0003CE7606A002801D004F0FAFC1C210B98E7
:106A00002AE7C0460C66FF1F10B5044C206800281A
:106A100003D004F0EDFC0023236010BD0066FF1FCF
:106A20000B4B07B51A68002A01D100200EBD69463C
:106A3000531C012012780731FFF772FC0028F4D0B4
:106A400002780123100018401A42EED0EEE7C0464B
:106A50001C66FF1FF0B51F4F01203B6887B0002B5D
:106A600025D09B78059300F0B3FB002821D00A20A5
:106A7000FFF7D4FA04000B20FFF7D0FA164B0500FD
:106A80001E78731E9E413B68F6B2191DD878FFF739
:106A900057FB3B682900DA7A043303929A79019311
:106AA0000292009033002000059A04F071FD07B0B7
:106AB000F0BDFFF7B5FF002805D00620FFF7AEFABE
:106AC00004000720D8E70820FFF7A8FA04000920EF
:106AD000D2E7C0460066FF1FFC65FF1F70B50A4E77
:106AE000040033780D00FF2B0DD0042004F058FB78
:106AF000011E08D0D0230370CE3B45708370C47054
:106B0000307804F02DFE70BD8044FF1F70B5040086
:106B100006200D0004F044FB011E0AD0D0230370B0
:106B2000CD3B8370054B44701B688580187804F05A
:106B300017FE002C01D0FFF767FF70BD0066FF1F36
:106B4000F8B5264F06003B680D001124002B05D137
:106B50000522234B1B78134202D112242000F8BDDA
:106B6000204A10241268002AF8D01278002AF5D0A2
:106B7000DB0719D52B789A1E012A1AD80C2004F0AD
:106B800087FD132438600028E8D000230A224370D0
:106B900029000670023004F0ABFBFFF75BFF041E18
:106BA0000AD0FFF731FFD9E700F012FB0028E1D14E
:106BB000E4E7002BE2D0D0E70B4B1B78032BCDD1C1
:106BC0001D20FFF72BFA094B18800028C6D0084B70
:106BD00004211878074A04F02BFDBFE70066FF1F69
:106BE000FD65FF1F1C66FF1FFC65FF1FFA65FF1F89
:106BF0002866FF1F60EA0000F7B50193194B1400E7
:106C00001A78052306000F0012201A4221D001290C
:106C100020D1154B1D68002D1BD002201F2C18D829
:106C2000002C02D0019B002B13D0104B1F221E7092
:106C30006E1C0021300004F033FB0199220030006B
:106C400004F056FB310020002C70002F06D004F019
:106C50003FFBFEBD064B12201D68DCE704F068FC1C
:106C6000F7E7C046FD65FF1F1C66FF1F8044FF1F3E
:106C70001866FF1FF8B50F4E12243368002B17D08B
:106C80001B780F3C834213D100250B4F022138782B
:106C900004F0A6FC094B042138781D8004F0A0FC08
:106CA000074B28001D8033685C7004F0C9FB0400AA
:106CB0002000F8BD0066FF1F2866FF1F1466FF1F37
:106CC000FA65FF1F70B5012823D11B4C2388002BC8
:106CD00003D01A4A1578002D07D0194B1B68002BDA
:106CE00002D01878FFF7C6FF70BD3B2B02D93C3BA2
:106CF0002380F9E7134E0221307804F071FCFA2268
:106D00002388920002215A43307804F0D1FB258079
:106D1000EAE70B4B1B68002BE6D00B4B1B785B079D
:106D2000E2D5084B0221187804F05AFC0022024BED
:106D30001A80FFF769FED7E71466FF1FF865FF1F8B
:106D40000066FF1F2866FF1FFD65FF1FF8B51E4D7B
:106D50002868002803D004F04BFB00232B601B4E57
:106D60003068002803D004F043FB00233360184F41
:106D700005243B7818002040234221D0154800F01C
:106D80002BFA3B78234213D0202004F081FC2860AA
:106D9000002813D02022002104F082FA202004F0E1
:106DA00077FC041E306005D02022002104F078FA20
:106DB000002004E0286804F01BFB2C601320F8BDC1
:106DC00000F00AFAF4E7C0461C66FF1F1866FF1FB2
:106DD000FD65FF1F7444FF1F10B50A4C23681A1E7F
:106DE0000ED0002808D10130587004F029FB00288B
:106DF00005D02368002B02D00021FFF787FE012277
:106E0000100010BD0066FF1FF7B5274E0500336860
:106E10000191181E21D05C78244F012C30D1FFF74E
:106E2000FFFD002825D02000FFF7F8F804004128D6
:106E300014D91F4B022118781E4A04F0F9FB1E4B8F
:106E40003C3C1C80022233685A703B78002B14D1E2
:106E500028000199FFF75AFE0120FEBDFA22920098
:106E60004243002AEED0124B0221187804F020FB96
:106E7000E8E7FFF7D3F80200F3E700233B70EBE706
:106E80003B78002BE8D1032004F08AF9011E08D0DA
:106E9000D0230370CC3B457083703368187804F0BE
:106EA0005FFCFFF7B1FDD7E70066FF1FF865FF1F26
:106EB0002866FF1F60EA00001466FF1F10B517491F
:106EC000838802008B4220D011D815498B4217D0FD
:106ED000144900205B1899B2012907D892681178EB
:106EE0005A425341D8B2FFF7F9FD012010BD0E4AB6
:106EF00000209B1807229BB29A424041C0B2F5E79E
:106F000083681878FFF768FFF0E7836899785A7804
:106F1000090218781143FFF777FFE7E70A2000001E
:106F200006200000F8DFFFFFAFDFFFFF014B187006
:106F30007047C0468144FF1F10B5064C207001F019
:106F400041FA207804F0C4FB0521207800F062FDAE
:106F500010BDC0462866FF1F0BB273B50D00002B95
:106F600000DBC4E0884B187804F0CAF9041E0ED088
:106F70000378912B0FD0A22B00D1A1E0834B18787E
:106F8000FF2852D0210004F0EBFB00284DD18020D7
:106F90000002684076BD43780F2B76D013D8052BBE
:106FA00070D00E2BEAD18088794B98422BD8794B40
:106FB00098421BD8784B9842E0D1A3681878591CA6
:106FC000FFF774F838E03E2BD8D18378032B74D0C8
:106FD0006CD8012B6ED0022BD0D1704B1B68002BCC
:106FE00023D05B68002B20D098471EE06C4BC01864
:106FF0000C28C3D804F034FB1DC2C2150BC20B0B06
:107000000B3223C23C00674BC0180728B6D8664B2A
:107010001B68002B09D01B68002B06D02000984766
:107020000AE0A3681878FFF7C7F8200004F0D0F949
:10703000ADE7A068FFF762F800289FD0F5E7A368E6
:107040001B78002BF1D0554B1B68002BEDD01B6833
:10705000002BEAD0210055489847EDE74F4B1B68BD
:10706000002BE2D01B68002BDFD021005048F3E753
:10707000504B1B68002BD8D05B68002BD5D021006B
:107080004348E9E7FFF7EAF9CFE780884A4B98429F
:1070900003D04A4B984200D070E7464B1B68002B48
:1070A000C3D05B68002BC0D02100D5E7153B012B76
:1070B000BBD963E7FFF798FAB7E7FFF77DFAB4E7C4
:1070C0003F4B1B78042B07D100236A4613800179BC
:1070D000408800F0C5FCA8E7364B1B68002BA4D005
:1070E0005B68002BA1D00100364898479DE701243A
:1070F00021420AD0294B1B68002B04D05B68002B6F
:1071000001D000209847012043E78B070AD5264B82
:107110001B68002B04D05B68002B01D0200098472F
:10712000022036E70421280008400D4200D131E753
:10713000254E3388002B21D0013B9BB23380002B9E
:107140001AD1FFF7DBF800280AD0204B1C70164B31
:107150001B68002B04D05B68002B01D020009847EF
:10716000FFF7C6F8694601F001FD6846FEF7FEFF2D
:107170001D20FEF753FF308004200AE7024B1878E9
:1071800004F02EFAF8E7C0462866FF1F8144FF1F6F
:107190000E20000001200000091000002066FF1FE3
:1071A000FEDFFFFFAFDFFFFF2466FF1F0C200000A4
:1071B0000B2000000866FF1F0D20000013200000B8
:1071C000FD65FF1FFFFF0000FA65FF1FF865FF1F49
:1071D00010B501F09BF910BD014B18607047C04617
:1071E0002466FF1F0B880020162B01D817230420CC
:1071F000014A13807047C046D265FF1F00207047C8
:10720000074A03001188814207D0918800209942E3
:1072100002D101308000101870470020FAE7C04604
:107220003066FF1FF0B58F7806000D00C7B01E2F27
:1072300015D1FFF7E5FF051E03D10024200047B05C
:10724000F0BD00223B003100C078009200F0B2FB9C
:107250000400A81C00F0D3FBFF23EB70EEE7264BE5
:10726000062403931B78FF2BE8D0182FE6D87B0861
:10727000224A013BDB0002929A589446002ADDD054
:10728000029AD3185B68002BD8D00878002802D166
:107290004B78012B02D10624122FCFD107AFAB8838
:1072A000697800976446AA68A047041EC6D1AB78E7
:1072B000029A5B08013BDB00D318390030005B68A1
:1072C0009847041E0BD1AB78042BB6D0039A31003B
:1072D00010782200009700F06DFB0400AEE76A789A
:1072E000002AABD1AA7805A93B88087130000A7042
:1072F0004B80FEF747FBA0E78444FF1F9CB90011B9
:107300001D4B37B5050098420BD000290AD1FFF775
:1073100077FF002805D11948FFF772FF002800D039
:10732000058037BD01291AD1FFF76AFF041EF8D086
:1073300001235B420380A378FF2BF2D0FE2B07D002
:107340000023E0781422009329001E3300F032FB62
:10735000A01C00F054FB01235B426380E1E702299B
:10736000DFD1013901F0BEF80028DAD12800FFF79B
:1073700047FF041EDFD1D4E7FEFF0000FFFF00003F
:10738000022210B5074B52421A80074801325A8038
:107390009A80DA8000F07EFA044801F025F8002097
:1073A00010BDC0463066FF1F257200110173001129
:1073B0000388F7B50400002B02D102252800FEBD8A
:1073C00042680221137825485268FEF7A5FD00287F
:1073D0002ED0234F01253A88002AEFD08023218820
:1073E0005B0201259B1A9942E8DC0C2004F050F95D
:1073F000061E31D03B8822889C4600231800019548
:1074000061469DB2491989B2AA421BD8002801D011
:1074100062443A8000233000082208C0210003F0B3
:1074200067FF104A1368002B13D100251660C5E7CB
:107430006268022113780C485268FEF76DFD00283F
:10744000C7D1BAE760681D01401941810133019835
:10745000D6E71A001B68E6E71325AFE70ABA001162
:107460008244FF1F2C66FF1F08BA0011014B1870E1
:107470007047C0468444FF1F14230A0010B51A4009
:10748000194204D00122102101F048F810BD4B062A
:10749000F9D4012088434000F8E710B514008B06AA
:1074A00004D50122102101F039F810BD08230A008B
:1074B0001A40194202D14BB2002B0FDA102101F011
:1074C0002DF8002808D02300F9331B78002BECD0CE
:1074D000F8342378012BE8D10020E6E70320890760
:1074E000FAD4E2E7F0B51F00184B85B01C68019094
:1074F00002910392002C27D1200005B0F0BDA568B1
:107500003301ED186B89019A934211D3029A934289
:107510000ED8002F04D10A9B002B10D12C00EBE7D2
:107520003B002978039A6868FEF7F6FC0028F2D140
:107530000136B6B2A388B342E1D82468DAE7A3687B
:107540000A9A5B891380E9E70026F3E72C66FF1FA0
:1075500037B50C000A8849880123914217D3002AC5
:1075600015D0651D23792A0002210A48FEF7D4FCB4
:10757000102300280BD023796188208800242A005A
:107580000094FFF7AFFF0A23A04200D023001800A9
:107590003EBDC0460ABA001113B50A0008884988E2
:1075A000012388420BD8002809D000241379053222
:1075B0000094FFF797FF0A23A04200D02300180091
:1075C00016BD13B50A0008884988012388420BD8E4
:1075D000002809D00024137905320094FFF782FFB8
:1075E0000A23A04200D02300180016BDF0B58BB0CE
:1075F00003904A8808880E000123824255D3002850
:1076000053D00023012704AC23700022718813009B
:107610000092FFF767FF051E3ED02078002835D185
:107620002B78022B18D167706A8983000130E31828
:1076300080005A8069680222201803F059FE2378DE
:107640000133DBB22370042B19D93B006889013068
:1076500080B2002BD9D01FE002236370122358435D
:107660006A89231804305A8069681022201803F0B0
:107670003FFE23780133DBB22370002BE5D10C4AA7
:107680006B899B185A425341DBB2DFE76378012BC9
:10769000E4D12B78022BC7D022780A23002A04D009
:1076A00021000398FEF798F9002318000BB0F0BDF5
:1076B0000100FFFF0F4BF0B504001868002816D03A
:1076C00083685D89A54207D88288AE18B44203DA80
:1076D00012019A18934201D10068EFE71E005F89FA
:1076E0001036A74204D1002900D00D801800F0BD4B
:1076F0003300EFE72C66FF1F70B505000C0008880B
:107700000021FFF7D7FF03000120002B04D0220047
:107710002800197AFFF7C1FE70BDF7B50C000025EF
:1077200001902300F6331B78AB4201D800200AE019
:107730006B00E65A00213000E718FFF7BBFF002876
:1077400002D126800130FEBD017A0198FFF794FE38
:10775000002802D03B882380F5E70135EDB2E0E751
:1077600010B5040008880021FFF7A4FF03000120E2
:10777000002B03D02000197AFFF77EFE10BD000019
:10778000054B1B68002B01D1180004E09A68528950
:107790008242F6D1988870472C66FF1FF0B50E27FD
:1077A000002687B0039302ABFF183E8005001F4BF5
:1077B00040891400984207D02B78013000976A68FE
:1077C00080B2FFF78FFE060002212B7818486A6806
:1077D000FEF7A2FB00280FD06C892000FFF7D0FF36
:1077E000002802D0013C0419A4B2039B002B00D056
:1077F0001C80300007B0F0BD02212B780D486A686C
:10780000FEF78AFB0028E7D102212B780A486A6834
:10781000FEF782FB002807D0002EDED03B88A34273
:10782000DBD17489013CDFE76C89DEE7FFFF0000F4
:107830000ABA001108BA001106BA001110B50C00FE
:10784000FFF7DEFC03000220002B0AD0002C00D042
:1078500023609B781720FE2B03D00138FF2B00D12B
:10786000002010BD73B50D0001A904001600FFF73C
:10787000E5FF172805D0002E04D129002000FEF7CF
:1078800027F976BD01221021200000F047FE0028D4
:10789000F3D0F6E7014B18607047C0463C66FF1F07
:1078A00037B56B469D1D010004000222280003F03D
:1078B0002FFF2B88B02B0ED12379122B09D1230057
:1078C000FF339B78012B06D10121608800F0E0F89E
:1078D00001E01B2BF8D037BD10B5054B0421187003
:1078E00000F098F8FFF74CFDFEF770FB10BDC046A6
:1078F0004066FF1F0020F0B50BB20F0087B0834237
:1079000034DA274B187803F0FBFC051E2BD00378E4
:10791000A02B25D103AE3100FEF7E4F8041E0BD1F5
:10792000B378DB0724D51F4B06341B68002B03D02C
:107930003100688898470400A868002801D003F047
:10794000F7FC002C08D1184A039B1340174A9342B6
:1079500006D0B3781B2B03D00121688800F098F87B
:10796000280003F035FD80200002784007B0F0BD0C
:107970000F4B1B68002B10D0310068889847041EFD
:10798000DAD07378002BD7D1B27801A90A704B8076
:107990000C716888FDF7F6FFCEE70624F1E7C046D4
:1079A0004066FF1F3866FF1F00FFFF000001120046
:1079B0003C66FF1FF7B50190822040000D001700C4
:1079C0001E0003F0EDFB04001320002C12D0B023A6
:1079D00020002370089BFC226770658026710830A8
:1079E000002B08D0190003F083FC2100019803F05C
:1079F000B7FE0020FEBD089903F052FCF5E710B574
:107A0000041E06D00078FD2803D803F029FCFF23CC
:107A1000237010BD0A1F93B210B504000220032B7F
:107A200005D882400020024BD1529B189C7010BD9B
:107A30006066FF1F0B8870B5043B04000D00022038
:107A4000032B0BD80121200000F04CFD0300142073
:107A5000002B03D02900200000F0DEFB70BD0000E9
:107A600007B51300034A00920A00012100F02CFC24
:107A70000EBDC0469D7C001107B501920322009205
:107A8000024B0A00122100F049FC0EBD1B7D0011C3
:107A900007B56B4601AA11800449D88008780633DF
:107AA000012802D1190003F05BFB07BD4166FF1FEF
:107AB0000C4B10B518700023FF210B4A1380138163
:107AC00093819380094A538013705172938193720A
:107AD000D174D3821375517703F022FE00F0FCF9C4
:107AE00010BDC0467066FF1F6066FF1F4266FF1F25
:107AF000F0B58DB06B46002003910C229B5E834253
:107B000000DBB0E05D4B187803F0FAFB051E00D1F6
:107B1000A4E00378902B00D09DE006AF01004688DA
:107B2000380000F013FA79680400002900D19CE0C5
:107B30003B88052B6ED13B89032B1CD905AC20005B
:107B400000F0A2F86288172A61D83989131D99427A
:107B500031D17968237804310291D90738D560781A
:107B600000F08EF9071E06D0002303712378012B45
:107B700008D0132B23D0A868002800D178E003F0A8
:107B8000D7FB75E06288029909A800F0A6F8029078
:107B9000380000F08BF909AA2378387A0192002284
:107BA00031000092029A00F012F9380000F064F9F6
:107BB000029B002BDFD0300000F080F9DBE7037878
:107BC000032BD8D16288029909A800F0D6F8DEE725
:107BD000122B13D1029909A800F0B5F8021EEAD1C0
:107BE00027498B88002BC6D0887909A92378019171
:107BF00061780091310000F0EAF8BCE7002302AAA6
:107C000093833000617809AAFFF72AFFB3E71D4B81
:107C10000993F6E7042B02D09A1F012AABD8184A21
:107C2000043B9B00995A0029A5D0D21890783100C6
:107C30003A0000F0AEF800289DD13B88042B03D019
:107C400001213000FFF724FF012C04D1A86800288F
:107C500001D003F06DFB280003F0BAFB8020039BEA
:107C60000002434018000DB0F0BD012800D182E7AA
:107C700001213000FFF70CFFEDE7C0467066FF1FE3
:107C80006066FF1F010017000B7803704B7843708C
:107C9000CB788A781B021343438070470A8803001D
:107CA00002700A88120A42700A88012A06D14A889C
:107CB00082704A88120AC2700420704702208242F1
:107CC000FBD14A8804309A704A88120ADA708A888E
:107CD0001A718A88120A5A71EFE710B50400012060
:107CE00082420CD94B780A781B02134323808342CB
:107CF00006D1CB788A781B0213436380002010BD25
:107D0000022BFBD1CB788A781B02134363804B791B
:107D10000A791B021343A380F0E70B8803700B88DA
:107D20001B0A43704B8883704B881B0AC3708B8877
:107D300003718B881B0A4371CB888371CB881B0A24
:107D4000C3710820704703000120082A14D14A7823
:107D50000878120202431A80CA7888781202024315
:107D60005A804A790879120202439A80CA7988793E
:107D7000120202430020DA80704710B5040001208F
:107D8000022A05D100204B780A781B021343238076
:107D900010BDF8B5060010200F00150003F000FA22
:107DA00004000120002C0ED0A0230C2229002380E7
:107DB0006780201D002D07D003F09AFA21003000C3
:107DC00003F0CEFC0020F8BD03F06AFAF6E7F7B541
:107DD0001E00009008AB142017001D78019103F0DD
:107DE000DFF9041E12D0A2230370019B4770438069
:107DF000099B057146710C220830002B07D0190031
:107E000003F076FA2100009803F0AAFCF7BD099967
:107E100003F046FAF6E737B5041E0FD04388002B6F
:107E20000CD00025C1881323007A172201950095F4
:107E3000FFF7CDFFFF2365806372257037BD00001B
:107E400010B50C4904004A88002A09D08B89002B00
:107E500005D00020CB8A0222834201D010BD01222E
:107E600013000A20434300204032C854C8184280FF
:107E70000472F3E74266FF1F0023438003707047DC
:107E8000094B00211A0010B55C88002C06D01C7923
:107E9000844203D10A234B43D01810BD01310A3369
:107EA0000329F1D10020F8E74266FF1F10B5040056
:107EB000407A03F0D5F9FF23637210BD7047043098
:107EC00010B580B203F064FA002803D004214942BF
:107ED00003F04EF910BD000070B50025104CA068ED
:107EE0002580A581A580A84202D003F021FAA560D3
:107EF00000250C4C0C4B606D1D80230058331D7009
:107F0000A84202D003F014FA6565002560680028D5
:107F100001D003F00DFA013508340A2DF6D170BDF9
:107F20000867FF1FAC66FF1FFC66FF1F70B5041ECD
:107F300009D1054D2880A881A880A868002802D012
:107F400003F0F6F9AC6070BD0867FF1FF0B54B8811
:107F500085B00193002343600A7905000F00022ACF
:107F600000D07BE0CA88032A17D98B685E7819781D
:107F70003602DC78D8790E4399781B7A24021B02EA
:107F80000C43034353495BBA0B80331D93421ED10C
:107F9000042C04D0631F022B0ED9012015E0019A96
:107FA0004D4B1201D35A002B06D00198FFF7BEFFAC
:107FB0004A4A1369013313610421B8682E812C8069
:107FC000494203F0D5F86860002005B0F0BD434D8C
:107FD000042C06D0631F022B0FD9EB680133EB6032
:107FE000DBE7019A3C4B1201D35A002B05D00198D4
:107FF000FFF79CFF2B6901332B61374B3000029355
:10800000019B029A1B010193002301998C468B521C
:10801000130063449C8003939E81FFF750FF039BF2
:10802000041E986016D00421B868494203F0A0F8F5
:10803000FA880100043A200003F05AF90199029AE3
:10804000FB888A5A043B9B18029A8B522B68013397
:108050002B60A2E7AB690133AB619EE71E4B029335
:10806000019B1E01029BF35A002B2DD002998C1903
:10807000A068002828D0012A26D1FA889B189BB234
:108080007352A189994217D39B1AC018B96803F09B
:108090002FF9029BA289F35A934200D07DE7002278
:1080A0002B81A3882B80A3686B60029BF2520B4A42
:1080B00053680133536070E7084A93680133936053
:1080C0000198FFF733FF68E7044A536901335361AE
:1080D000F6E7C0467266FF1F0867FF1F7866FF1F3E
:1080E00070B5051E15D10B4C0B4B1880230058336F
:1080F0001870606D002802D003F01AF9656525003C
:1081000050356068002801D003F012F90834AC4201
:10811000F7D170BDAC66FF1FFC66FF1FF0B51700FE
:10812000A12285B0920001934243394B06001B689F
:108130000C009B18D933FF331D78FDF741FF043045
:10814000854204DD3000FDF73BFF0430C5B2BD427F
:1081500007D33A0000213000019B03F079F905B004
:10816000F0BD2900380003F0A3F82300C6B2503355
:108170001E700393019B29006365380003F000FB28
:10818000CBB20293002B02D0039B01361E70002657
:108190002300503303931B78B34204D8606D00284A
:1081A00031D10020DBE7029A2800002A04D0013BED
:1081B0001000B34200D02800F700E719387003F030
:1081C000C7F8786000280ED03A78019903F090F84B
:1081D000019A3B780136D3180E4A0193D369F6B25F
:1081E0000133D361D4E7039B18706065A74205D1C2
:1081F000084A1320D36A0133D362B0E7606803F002
:1082000097F80834F2E703F093F800236365C8E7B2
:108210003409FF1F7866FF1FF7B50D000700042122
:10822000686802F0A5FF2B89040003702B891B0AE4
:1082300043702B8883702B881B0AC3702E890225FC
:108240000436F6B2FB2E15D81B4B9F4214D10C20DE
:1082500002F0A6FF1135011E0CD0902303708E3B57
:108260000371043B4380154B8460C680187803F08B
:1082700077FA00252800FEBD5C237B43104AD31803
:108280000093583301931B78002B0FD10300320069
:1082900038000099FFF742FF019B05001B78002B77
:1082A000E8D13800009903F01BF8E3E7054A0725F9
:1082B000536A01335362DDE7FEFF00007066FF1F63
:1082C000AC66FF1F7866FF1FF0B587B000901720DF
:1082D0000F0016000193FFF7F2FD1325041E19D0BD
:1082E0000C98031E02D00199201D9847030AE370E1
:1082F000052302AAA0700430908127700098667050
:1083000003A993800494FFF787FF051E02D0200085
:1083100003F00EF8280007B0F0BD0000F0B587B0FC
:108320001F000CAB1B780391059301210DAB0600D8
:108330001C78049200F0D6F81425002821D02000E3
:10834000FFF77EFD0135041E1BD01149059B0A78FD
:1083500003700132D2B2131EC68001D101231A006C
:108360000B7022713000049B03990097FFF7ACFF5C
:10837000051E09D1230021000648074A093303F0EE
:10838000E7F9280007B0F0BD002363802370F8E709
:108390007466FF1F177E001130750000F8B50500E8
:1083A0000E00064C064F2368002B02D03100280037
:1083B00098470434BC42F6D1F8BDC0461867FF1F89
:1083C0002C67FF1F0123064A5B4253800023137171
:1083D0005362044A136053609360D3601361704723
:1083E0002C67FF1F1867FF1F0200002310B5064906
:1083F0009C000859002801D1625010BD0133052BA3
:10840000F6D11320F9E7C0461867FF1F034A5388C7
:10841000181A434258414042104070472C67FF1FD2
:10842000F0B585B002930AAB1F780CAB1B880090A7
:1084300008000E0001920393FFF7E8FF05001120EA
:10844000002D1BD10E48FFF7E1FF04001520002C82
:1084500014D006220B99A771E01D02F049FF019B81
:1084600030002371029B29006371009B668023709A
:10847000039B6562E381FFF791FF280005B0F0BD23
:10848000FFFF000010B5FFF7C1FF04000220002C21
:1084900012D060880121FFF781FF606A002801D0B7
:1084A00002F0A6FF28220021200002F0F9FE01239D
:1084B00000205B426380207110BD000030B5074A88
:1084C000074C5588010013780020A54204D05B1AA0
:1084D00059424B415842104030BDC0462C67FF1FE7
:1084E000FFFF0000084A10B501230C00904208D09D
:1084F000FFF78CFF031E04D0037923405A1E9341DB
:10850000DBB2180010BDC046FEFF0000024B187918
:10851000431E9841C0B270472C67FF1F70B504001E
:108520000D001600FFF772FF002804D10D4B9C428E
:1085300000D0143070BD416A03790520002907D0AE
:1085400012221A40102A02D10520002EF2D10F204B
:10855000DB06EFD5897E0C20A94289414942494278
:108560000840E7E7FEFF0000030010B5002800D137
:1085700010BD0348034A41889142F9D09847F7E774
:108580002C67FF1FFFFF0000002330B5C45CCD5CEB
:108590006C40D4540133102BF8D130BD0F2300228E
:1085A00010B5C45C64002243CA54C25CD209013BCA
:1085B000F7D210BD0200010010B52032103102F0D8
:1085C000F7FD10BDF0B58BB0039010200593170098
:1085D000049103F05DF80090102003F059F8009B1F
:1085E00013240190002B05D000280CD113240098EF
:1085F00002F0FEFE019B002B02D0180002F0F8FEF4
:1086000020000BB0F0BD102003F042F8060010204F
:1086100003F03EF813240500002E00D1AEE0002840
:1086200019D01022002102F03BFE320029000398ED
:1086300002F0BEFD041E0ED133787F2B51D83000DE
:108640000099FFF7ABFF009B1B787F2B53D8019954
:108650000098FFF7A3FF300002F0CAFE002D02D001
:10866000280002F0C5FE002CC1D1102003F010F844
:108670000600102003F00CF80290002E7CD0002899
:1086800078D03A000F3223000125121105D00F33A4
:108690003B4015B25A4253411BB26A1E1201002BD5
:1086A00033D0049BD2B298180099029AFFF76CFF5E
:1086B000013D10220021300002F0F2FDADB2049F16
:1086C0002D017D19AF4242D0002C33D0300002F092
:1086D0008FFE029B002B00D189E7180002F088FE74
:1086E00085E729003000FFF759FF28002549009A47
:1086F000FFF74AFFA7E729000098FFF74FFF280080
:108700002049019AFFF740FFA5E70F210F40049988
:108710008A18D9B28F4208D9D15C06A819540133FE
:10872000102BF6D1029A0199C0E7791A48424141CB
:10873000C901F2E73900300006AAFFF725FF320031
:10874000039806A902F034FD10370400BAE7002CA4
:10875000BCD13000029906AAFFF716FF320006A925
:10876000039802F025FD082204003100059802F06C
:10877000BFFDABE71324A9E71324AAE7002800D024
:108780006EE733E710BA0011F0B58BB00F0016009A
:108790000225009000283FD0002A3DD00B1DDBB2FF
:1087A0001800029302F074FF1135041E34D0FDF757
:1087B00047FD05003A000099201D02F021FDEBB2B3
:1087C0000393E3702B0CDBB22F0A00936370FFB2AC
:1087D0002B0E2370A7700193FDF72CFD10220100D2
:1087E00006A802F00DFD2100029A04AB06A8FFF7CF
:1087F000E9FE051E0DD1039B08223370009B04A9DE
:10880000B370019B7770F370301D02F0F9FCFDF737
:108810001DFD200002F0ECFD28000BB0F0BDF0B50E
:108820008FB00D00149E039004920593002A03D18B
:10883000022420000FB0F0BD002EF9D00398FFF7FE
:10884000E5FD1424071EF4D07278337812021A431F
:10885000B3781B041343F27812061A43036A019299
:10886000934201D30133E3D1002D03D03B7901249E
:108870009B07DED50822002106A802F011FD059B0A
:1088800013240433DBB21800029302F001FF051E2B
:10889000CFD0059A0499043002F0B2FC04223100D2
:1088A000280002F0ADFC3900102210310AA802F0B5
:1088B000A7FC2900029A06AB0AA8FFF783FE041E54
:1088C0000FD1082206A908A802F09AFC0822311D3F
:1088D00008A802F0CDFD012807D101990398FDF702
:1088E000C9FC280002F084FDA3E70124F9E7000099
:1088F00070B51C4C05002368181E10D0002D14D133
:108900001A78002A0CD1981C083202F0F1FC02F00F
:1089100057FC0135002808D123681D70012070BD67
:108920000A331800082202F0E3FC2368002BF5D07C
:10893000122002F035FC061E0DD0C1232168037001
:10894000457002311022023002F0D2FC236831005F
:10895000587802F005FF206802F04AFD00232360EA
:10896000DCE7C0465467FF1FF8B504002020FDF780
:1089700055FB0D4EA700BB590500002B0DD000285C
:108980000BD0D878FF2809D108492A000C55F35993
:1089900007480333611802F0DBFEF8BD290002F03E
:1089A000EFFC0028F0D1F8E77067FF1F5867FF1F42
:1089B000C19B001170B5064D84006359002B05D092
:1089C000D87802F04DFCFF226359DA7070BDC046C2
:1089D0007067FF1F70B506008CB00C0015000021F9
:1089E0003022684602F05CFC31001022684602F03A
:1089F00007FC1D2021000322684402F001FC6846A8
:108A0000FFF7D8FD2D21040003222800694402F05D
:108A1000F7FB20000CB070BDF0B50700160097B052
:108A200001931CAB1D7830221EAB00910AA80021D7
:108A30001C7802F035FC102239000AA802F0E0FB95
:108A40001022002102A802F02BFC0722310002A80C
:108A500002F0D6FB072202AB9818631E9C410199D5
:108A600002F0CEFB02AB9C732B005A1E934102AA6C
:108A7000D3730021102206A802F012FC06221D99D1
:108A800007A802F0BDFB1A2002ABC01806221F99EE
:108A900002F0B6FB102200990EA802F0B1FB1022E2
:108AA00002AB0EA908781C78013A6040D2B2087077
:108AB00001330131002AF5D10AA8FFF77BFD10220E
:108AC00012A904000EA802F013FC102206AB0EA996
:108AD00008781D78013A6840D2B20870013301313C
:108AE000002AF5D10AA8FFF765FD0443102220985B
:108AF000E4B212A902F084FB200017B0F0BD70B5FB
:108B00000E0014008CB00100102268461D0002F017
:108B100077FB3100082204A802F072FB2100082232
:108B200006A802F06DFB6846FFF744FD0400102222
:108B3000280008A902F064FB20000CB070BDF8B555
:108B400006000D0000243719AC4200D3F8BD02F036
:108B500077FB030A3B70631CDBB201379D4203D9EC
:108B60000234F054E4B2EEE71C00EDE773B5060002
:108B70000C000225002819D0002917D0032101A8D4
:108B8000FFF7DDFF6B469A793F231A400133134309
:108B90006A463000937101A92200FFF71BFF051EF2
:108BA00004D10322E01C01A902F0A2FB280076BD3B
:108BB00003785807DA08C00FD20080009B071043E3
:108BC0009B0F1843C0B2704707230B40C908C90068
:108BD0000B4303707047000070B50400FFF7EAFE16
:108BE000134DA4006359002B21D0186A002801D02E
:108BF00002F0FEFB2B59986E002801D002F0F8FB22
:108C00002B59D86E002801D002F0F2FB2B59186FB7
:108C1000002801D002F0ECFB2B59586F002801D03E
:108C200002F0E6FB285902F0E3FB00232B5170BD54
:108C30007067FF1F0E4B8000C35870B50C00002BEF
:108C40000FD09D68002D0CD02B78201D0B706B78F9
:108C50004B70A97CFFF7B8FF2B7E23726B69E36032
:108C600070BD10220021200002F01AFBF8E7C04678
:108C70007067FF1F014B18607047C0466C67FF1F8D
:108C8000074A03008000825810B5002A06D0D08819
:108C9000984203D1012901D1FFF79EFF10BDC046C4
:108CA0007067FF1FF0B5264E95B087000B93BB5938
:108CB0000500099112200A92002B31D0D888FFF7C5
:108CC000A5FB04001420002C2AD0280010A9FFF7CF
:108CD000B1FFBB591E781D6A002E23D00895FDF701
:108CE000EFFA07000020FDF7F1FA0790A379E61DDF
:108CF000069310AD0CA9089800F0E2FA0EA928001E
:108D000000F0D7FA0B9B0A990493069B09980293EB
:108D1000079B0396019300970EAB0CAAFFF77CFE0E
:108D200015B0F0BDFDF7CCFA06903000FDF7CEFA95
:108D3000E31DA779079310AB06000893DAE7C04656
:108D40007067FF1F30B50C4C85002A59030085B0B1
:108D50000120002A0ED018006946FFF76BFF2B593F
:108D60001A78D888054B002A00D1054B6A4607219E
:108D700000F0D9FB05B030BD7067FF1FB392001142
:108D8000C192001130B5094C8500295985B01022D7
:108D90006846253102F0ACFA2A591121044BD088DB
:108DA0006A4600F0C0FB05B030BDC0467067FF1FCB
:108DB0005D93001130B5094C8500295985B010220A
:108DC0006846353102F094FA2A591121044BD088B3
:108DD0006A4600F0A8FB05B030BDC0467067FF1FB3
:108DE0009B930011F7B54D4F86001020F4590D00EC
:108DF00002F04EFCF3592062186A132200286CD04E
:108E0000033A29009C6802F073FAF3591A78019228
:108E1000002A58D11E6A227D317B9446514001229E
:108E2000019F114201D167461740217D914339438B
:108E30002175377B4F40BC4660460027800701D430
:108E40004F081740012102208F40227D82433A4380
:108E50002275377B5740BC4660460027400701D447
:108E600097080F400420227DBF0082433A432275B9
:108E7000627D002794466046727B42400A4201D1DF
:108E800067460F400121627D8A433A436275777BD2
:108E90005740BC4660460027800701D457080F4062
:108EA0000220627D7F00824317436775767B002234
:108EB0007E40760701D4BA080A400426617D9200FC
:108EC000B1430A4362756A78002A08D06278002AA2
:108ED00005D005220533DA7700221000FEBD0422FA
:108EE0002979114205D1A17C114202D10533033AFF
:108EF000F1E7019A21782C78002A02D10A0021009A
:108F0000140018220429E8D8042CE6D80520604370
:108F1000034A05331218525CDDE7C0467067FF1F35
:108F200020BA001110B50A001121024B00F0FBFA23
:108F300010BDC046F79300110B0030B587B001ADEE
:108F40002B806B4604001100981D082202F0D0F916
:108F50002A000B212000024B00F0E5FA07B030BDDB
:108F60001F94001110B50A001121024B00F0DBFA2A
:108F700010BDC0467394001113B50B0011006A4672
:108F800013706B4604000622581C02F0B1F96A46C1
:108F900008212000014B00F0C6FA13BD9394001184
:108FA00010B50A001121024B00F0BDFA10BDC046F9
:108FB000E39400117FB505000B4BAA00D4580800BC
:108FC000002C0FD0666F237FE28821780396266FEE
:108FD0000296E66E0196A46E0094FDF709FC280047
:108FE000FFF7FAFD7FBDC0467067FF1F10B5172160
:108FF000FFF7E0FF10BD000070B50A000D00064B42
:109000000221040000F08FFA060029782000FFF703
:10901000D1FF300070BDC046C393001170B586B05B
:1090200000236A461370836804001D78681E0A28AE
:1090300059D801A902F0ECF9060633373B3F434704
:109040004B4F5300180000F042F9062312284BD072
:1090500000281BD16088FFF7D9F90823002813D016
:109060004279002A47D1264B1A78072312070BD5DD
:10907000244B1A680723002A06D01668002E03D056
:10908000290001AAB04703006A4613706B461B789B
:109090006088002B2AD1FFF767FC06B070BD18006E
:1090A00000F06CF9D4E7180000F087F9D0E7180059
:1090B00000F093F9CCE7180000F0ADF9C8E718000C
:1090C00000F0C3F9C4E7180000F0F6F9C0E7180093
:1090D00000F0F6F9BCE7180000F013FAB8E7180042
:1090E00000F013FAB4E707236A46137069466088F4
:1090F000FFF782FFD1E70523012AC5D1024BB8E76C
:10910000FD65FF1F6867FF1F6C67FF1FF8B52C4FD9
:109110008600F35904000D00002B40D0DA8882420B
:109120003DD15A78062A33D11A78002A2ED0012050
:1091300099681A6A097D014206D0157B054203D061
:1091400007225A700120F8BD0220014204D0157B8D
:10915000054201D00922F4E70420014204D0127B29
:10916000024201D00B22ECE7164B1B68002BE9D022
:109170005B68002BE6D020009847BB5900215B7844
:10918000122BDFD12000FFF715FFDBE70E4BECE7DA
:10919000112A04D1002900D032252900F2E7002D40
:1091A00008D12000FFF732F9002803D010230279FC
:1091B0001343037121002800FDF798FAC2E7C04667
:1091C0007067FF1F6867FF1F6C67FF1F70B50E4E4B
:1091D0008500AB590400002B13D01B78002B11D154
:1091E0000A4B1B68002B04D05B68002B01D02000C9
:1091F000984773595B78122B03D100212000FFF7A9
:10920000D9FE70BD024BECE77067FF1F6C67FF1F54
:109210006867FF1F094B8000C3581020002B0CD03B
:109220001A6A002A09D09B68002B06D0127A1B7E8E
:10923000101C9A4200D9181CC0B270477067FF1FFB
:1092400070B503000D0014000220002A30D0002960
:109250002ED013700B78081D53704B789370FFF766
:10926000A7FCE070012002212B7A23716B7B034065
:1092700063716A7B0A401343042263716E7B16405C
:10928000334363716E7BF608F600334363712B7BC7
:109290000340A371287B014000200B43A371297B6D
:1092A0000A401343A3712A7BD208D2001343A3714F
:1092B00070BD10B50A0001000120FFF7C1FF10BD0D
:1092C00010B50A0001000220FFF7BAFF10BD70B50B
:1092D00006000C000220002E30D000292ED073781A
:1092E000201D0B70B3784B70F178FFF76DFC0122F5
:1092F0003579257271794B10080013409340104066
:109300000343881010408000C9080343C9000B4381
:109310006373B1794B10080013409340104003432E
:10932000881002409200C9081343C9000B43212052
:109330002373FCF773FE854201D2122070BD2220F8
:10934000257AFCF76BFE8542F7D823781820042B8A
:10935000F4D86378012BF1D80020EFE7030010B5B3
:109360000220002909D0002B07D00322481C0A70D4
:1093700019000D3201F0BCFF002010BD03000222D5
:10938000080010B5002B06D0002904D00E32591C5D
:1093900001F0AEFF0022100010BD030010B5022046
:1093A000002909D0002B07D00422481C0A7019009C
:1093B0000C3201F09DFF002010BD10B5FFF7DEFF5D
:1093C00010BD03000220002906D0002B04D0052286
:1093D00000200A701B784B70704703000220002B9E
:1093E00008D0002906D05B7800200B70013B082BC9
:1093F00000D918307047030010B50220002909D0A9
:10940000002B07D00622481C0A7019000A3201F00E
:109410006FFF002010BD10B5FFF7B0FF10BD0200B8
:109420000B00022010B500290ED0002A0CD0072115
:109430001970118859701188090A99701118082239
:10944000D81C01F055FF002010BD03000A000220C7
:1094500010B5002B0CD000290AD099785878090251
:1094600001431180901CD91C082201F041FF00200B
:1094700010BD030010B50220002909D0002B07D031
:109480000822481C0A701900921801F031FF0020D0
:1094900010BD02000B00022010B500290BD0002ADD
:1094A00009D009211970117818185970511C062219
:1094B00001F01EFF002010BD10B5FFF75FFF10BDCB
:1094C00002000B00022010B5002A09D0002907D0A5
:1094D0005178197011180622581C01F009FF00205C
:1094E00010BD030010B50220002909D0002B07D0C1
:1094F0000A22481C0A701900063201F0F9FE002009
:1095000010BD10B5FFF73AFF10BD02000B0002209E
:1095100010B5002A06D0002904D018005178FFF7B2
:1095200053FB002010BDF0B585B017001E006A4641
:1095300006230500080091819380FEF7C0FC1324E8
:10954000011E02900CD03800B047041E05D128003F
:1095500001A9FEF76FFA041E02D0029801F0E8FE9E
:109560002800FFF701FA200005B0F0BDF0B50400B7
:109570008BB0019115000021102202A801F090FE8D
:10958000334EA700B85900283CD0C388A34239D134
:109590000378002B36D14278062A18D10200010048
:1095A000553235310C3006ABFFF7A9FA002829D126
:1095B0002000FFF72FFE020006A902A801F098FE86
:1095C000200002A902F02CF801200BB0F0BD816E42
:1095D000002917D00B8A112A28D19D420ED101985B
:1095E0001231093A01F044FF012807D1BB5920008C
:1095F0009D6EFFF70FFE29000200DEE732212000FA
:10960000FFF7D8FC2000FEF701FF061E1BD0416AC1
:10961000002918D00B8AAB4215D1082201981231CB
:1096200001F026FF01280ED1716A0AE09D42E9D1BE
:1096300008220198123101F01BFF0128E2D1BB5929
:10964000996E8A7EB9E7200002F002F8BCE7C046B6
:109650007067FF1FF0B56B4D87007E5985B033787A
:1096600002900393002B00D087E0B368346A019323
:109670007078062817D101221B7D134202D0217B6E
:10968000114218D10222134202D0217B114251D142
:109690000422134203D0237B134200D08BE0019BB2
:1096A0005A7DEB5991E007380428F8D801F0B0FE54
:1096B000032E42678300B36E002B03D11C2001F000
:1096C000E7FFB066EB599C6E002C1CD010220021E5
:1096D000200001F0E5FD0298FFF79CFD010020004D
:1096E000FFF72DFA01F0ACFD208220000821123096
:1096F000FFF725FA0298FFF78DFDA076EB592100C0
:10970000D888FFF70FFC0822EB591CE0B36E002B42
:1097100005D01A00198AF0881232FFF70DFC0222D8
:10972000019B197DEB5911423DD0207B10423AD06C
:10973000073208E0F488FCF7DBFD01002000FFF7AA
:1097400011FC0A22EB595A70029B9C002A5953784B
:10975000073B042B11D8D088FEF758FE00284ED0C6
:10976000C3895A08D2182849029B0298CB542B5916
:1097700041180433254801F0EBFF05B0F0BDFCF7BC
:109780009FFD03000120834201D100200393EB5988
:10979000DE88FCF79BFD039902003000FFF7ECFB2D
:1097A000019AEB59117D042211420CD0217B114208
:1097B00009D00B22C7E7F688FCF73CFD010030001A
:1097C000FFF7EEFB6BE7019A527D01210A4204D0BC
:1097D000607B084201D00C22B5E702210A4204D086
:1097E000607B084201D00E22ADE704210A4204D07A
:1097F000627B0A4201D01022A5E71222A3E7FA22D7
:109800005200B0E77067FF1F7467FF1FCB9B00110A
:1098100010B5064B1A780423100018401A4200D0E5
:109820000348FFF727FA002010BDC046FD65FF1F63
:109830008844FF1F70B50400FFF7D4FA051E43D11A
:109840002000FFF77FFA234EA400A0598268937C82
:10985000DB0708D50321036A1B790B40012B02D1DA
:10986000017F0B430377431DD97F8B1E022B0DD83D
:10987000022900D00121C088FCF790FF0421335950
:109880001A7F59700A431A77280070BD01290CD13C
:1098900002231022437000210C3001F001FD3059E9
:1098A00010213530FFF74BF9EEE70529ECD1022303
:1098B000D118437010220C3001F01AFD04233259E4
:1098C000117F0B431377EAE708251828DCD1053D03
:1098D000DAE7C0467067FF1FF0B58BB0059143888B
:1098E0007E4F9E00F45915000493002C15D10129D8
:1098F00002D000200BB0F0BD101D57781678FFF78E
:1099000057F9EB68320002932B7A04990193009087
:109910003B002000FCF70CFFEBE7E388049A93423E
:1099200001D00820E6E72378012B00D1D4E0059B85
:10993000581E092800D9CFE001F06AFD05CE0A299A
:10994000CC506C859AB229000498FFF773FFD1E7D9
:10995000200029001022453001F0CAFCB9594B788B
:10996000042B02D1013B4B70C3E70B000A002533E7
:1099700035320C310498FFF795F90498FFF702FA95
:109980000522431E9841BB59C0005A70B2E720001F
:1099900029001022553001F0ABFC049B4F4C9D0078
:1099A000295904980A0006AB55320C31FFF77AF9B1
:1099B00029591022453106A801F05AFD012808D185
:1099C0000498FFF7F7F90590002804D106222B59D7
:1099D0005A7005988EE708230593FAE763780C2BF5
:1099E0007AD1E36E002B03D11C2001F051FEE0661A
:1099F000BB59D86E00286FD01022290001F078FCE6
:109A0000BB590498DC6EFFF705FC0D22A076BB590C
:109A10005A706EE7E06E00285ED063780D2B5BD144
:109A20002B8808220382A91C123001F061FCBB596B
:109A30009A68517D0222114226D0186A407B10425A
:109A400022D00C32E4E763780E2B45D1236F002B34
:109A500003D1162001F01CFE2067BB59186F0028A7
:109A600003D01022290001F043FC0F22BB59CFE79D
:109A700063780F2B30D1206F0622691C103001F063
:109A800037FCBB599A68517D0422114203D0196AF0
:109A9000497B1142D5D100210498FFF78BFA28E7C2
:109AA000636F002B0DD0BB59586F0028F3D01022E4
:109AB000290001F01DFC0122BB5952425B6F1A6163
:109AC000E9E7142001F0E4FDBB5960675B6F002BF0
:109AD000E9D126E72978DFE707200BE77067FF1F4A
:109AE00010B5064C207001F013FB06212078FDF71D
:109AF00091FF0348FEF778FC10BDC0468367FF1F47
:109B0000818C001100200BB270B50D00834216DA73
:109B1000264B187801F0F4FB041E0DD00378922B2D
:109B20000ED0A02B37D0224B1878FF283AD0210036
:109B300001F016FE002835D180200002684070BD7B
:109B400043780E2B0BD03E2BEDD18378052B12D012
:109B5000082BE8D181798088FFF7D8FA08E0154B07
:109B600082889A42DFD183681878591CFEF7C0FEBC
:109B7000002817D1D7E7104B1B785B0712D50F4B86
:109B80001B68002B0ED09B68002B0BD0C289811D57
:109B900080889847ECE7FFF741FAA068002801D0D9
:109BA00001F0C6FB200001F013FCC5E78367FF1F2F
:109BB0008144FF1F18200000FD65FF1F6C67FF1F19
:109BC00010B50078FFF712FA10BD10B50078FFF756
:109BD000FDFA10BD0C234343084A10B59B185A6880
:109BE000002A03D0012901D1904710BD9B68002BAA
:109BF000FBD00029F9D19847F7E7C046A067FF1FBF
:109C000010B5162813D801238340094A946B1C43CE
:109C10009463506B98435063D46B200098430129A0
:109C200001D120001843D063116B0B43136310BDA7
:109C300000800040F0B500240127154B85B0DA6B99
:109C4000144E03921A6C0192DA64019BE3403B428A
:109C500017D0039DE5403D400295E5B202992800EA
:109C6000FFF7B8FF316A736A002908D03900002B6A
:109C700001D0029979402800FFF7C2FF01E0002BD4
:109C8000F9D101340C36172CDFD105B0F0BDC04638
:109C9000008000408467FF1F10B5012402002000EF
:109CA000162A08D8054B5968D140214204D01868BB
:109CB000D0400123184010BD186DF9E70080004026
:109CC000162807D80122064B8240002903D0D96804
:109CD0000A43DA607047D9689143D960FAE7C04611
:109CE0000038004030B5162818D8032444430F4BE1
:109CF000E25C1B199C785D7801232D1B0135AB407C
:109D0000013BA340A140DB430C00122807D80849BF
:109D100092005218116819402143116030BD054A64
:109D200011680B4023431360F8E7C04667BA00117F
:109D300008F0004014F00040C21F70B5D4B20623F2
:109D4000092C0BD80125084C9540002908D000218A
:109D5000FFF7C8FF23682B4323600023180070BD62
:109D60002368AB43F8E7C04600380040F0B516283A
:109D700026D8214B1B185B78022B21D103244443A6
:109D80001E4A1F4EA35C12199478012215008540CB
:109D9000B76B013CE4B23D43A240B563194C1228B5
:109DA00015D89B0000290CD117495B1899680A4304
:109DB0009A600123205C154A834011680B431360AD
:109DC000F0BD11495B18996891439960F1E70E4B1A
:109DD00000290DD159690A435A61225C1328E8D041
:109DE0000123203A93400A49086803430B60E7E7E0
:109DF000596991435961F0E78467FF1F67BA001101
:109E000000800040ACBA001100F00040A0F000401B
:109E1000A4F00040F8B500241B4E1C4D1C4B1B5DEC
:109E2000012B1FD1184A9269E2401A420BD001223D
:109E3000AA5693402200143AD2B2022A09D81549F0
:109E40004A6913434B6101340C360235172CE5D1B6
:109E5000F8BD0022AA560F499200521891680B4390
:109E60009360F0E7022BEED1E7B23800FFF714FF62
:109E700001235840C1B23800FFF778FF3800FFF7E0
:109E80000BFF7077DFE7C0468467FF1F39BA001108
:109E90008567FF1F00F00040012202388240054B19
:109EA000002903D059690A435A617047596991439F
:109EB0005961FAE70038004070B504000D00052034
:109EC000162C1AD800212000FFF7FAFEA31E012B42
:109ED00003D801212000FFF7DFFF00212000FFF75A
:109EE0002BFF01220A49A2400A4B4868012D05D1E7
:109EF00002431B194A605D70002070BD90434860AA
:109F000002211C196170996991439961F4E7C04677
:109F1000008000408467FF1F10B516280AD8012270
:109F2000074B8240002906D019680A431A600121B4
:109F3000FFF7C2FF10BD196891431960F7E7C046EB
:109F40000080004070B505000520162D17D80C23A1
:109F500000246B430A4A21009B181C70094B2800FF
:109F60005B195C70FFF7A8FF0123AB402000064996
:109F70000A681A430A6005490A689A430A6070BD74
:109F8000A067FF1F8467FF1F3480004030800040BF
:109F900070B504000E00FF2813D003250540FFF71D
:109FA000D1FF084AA3089B009B183F22ED00AA405E
:109FB000AE40196820009143314319600121FFF739
:109FC0007FFE70BD18380040F8B505000520162D3D
:109FD00025D80C246C43124BE4186368002B03D182
:109FE000A3680D30002B1AD0022201270D4B00214F
:109FF0005B195A7028002770FFF75EFF63681E1E0A
:10A0000008D0A3683E00002B04D02800FFF744FED0
:10A010004640F6B228003100FFF7F2FD0020F8BDFF
:10A02000A067FF1F8467FF1FF7B5C420FF222B4BDB
:10A0300080001958002491437F3A0A431A50802225
:10A04000274F5202274E1A60274B1D5D002D21D04D
:10A05000A31E012B03D80121E0B2FFF71DFF012D44
:10A0600018D11F4B9B69E3402B4213D0E3B2180079
:10A070000193FFF711FE01000198FFF74DFFE3B2D6
:10A08000143B022B1DD801217156184A8D4053698B
:10A09000AB4353613B7F002B0DD0E5B22800FFF7A7
:10A0A00093FF2800FFF7F8FD7B7F0100834202D079
:10A0B0002800FFF78FFD01340C370236172CC3D16F
:10A0C000F7BD012100237156F3568D40074A9B00CE
:10A0D0009B189A68AA439A60DCE7C04600E100E05A
:10A0E0008467FF1F39BA00118567FF1F00F0004029
:10A0F00010B504000520162C0CD801212000FFF714
:10A10000DBFE0123044A002011194B70A340916922
:10A110000B43936110BDC0468467FF1F70B50E00EE
:10A1200015000400FFF70EFF0C236343094A2000CB
:10A130009B189D605E60FFF747FFF021064B074AC2
:10A140008900051E5A5002D02000FFF7FBFE2800B0
:10A1500070BDC046A067FF1F0000FF1F359C0011A7
:10A1600070B5134D07202C78002C1FD198222100A8
:10A170005200280001F02CFA0123C420FF222B708A
:10A180000C4B80001C635C630B4B1C605C600B4BD6
:10A19000195891437F3A0A431A50802252021A609A
:10A1A0000D20074A074901F0CBFA200070BDC046D8
:10A1B0008467FF1F00800040A0F0004000E100E045
:10A1C00029A00011159E0011030010B50620072BD1
:10A1D00009D8054A137001F0A3F9D7210020034BD9
:10A1E000034A89005A5010BDB044FF1F0000FF1FF2
:10A1F000151BFF1F70B51D0002240C2910D8094A39
:10A20000CA40D2070CD5FBF715FF041E08D1059AEA
:10A2100004992800FBF72AFFFCF798FDFFF7F8FAEE
:10A22000200070BD1210000030B50D7802232C0004
:10A230009C43184201D02B431C0008252300AB434C
:10A24000284201D02B00234320241D00A543204297
:10A2500001D01C4325002A230D70184204D0117828
:10A260001E3B0B43137030BD0028FCD10C2113782A
:10A270008B43F7E7F8B51D0006AB1B88140007AA4F
:10A280000E000B201778002B27D10A78022A49D11B
:10A290004A68507811780002244A0843801804283C
:10A2A00040D801F0B5F803121D1B2300F06801F03F
:10A2B0002FF9021CC0B2B84200D93A1CD2B2200019
:10A2C000F1682A8001F014F806E00222F3681B8886
:10A2D0002A8023701B0A63700020F8BD0622EEE777
:10A2E00001232B80F3681B782370F5E7F368002BBC
:10A2F00016D008222A801A8822701A88120A6270E0
:10A300005A88A2705A88120AE2709A8822719A8832
:10A31000120A6271DA88A271DB881B0AE371DBE73B
:10A320002B80D9E701202B80D7E7C04600D6FFFF5E
:10A33000F7B516000A781D0008AB1F880C00012332
:10A34000022A18D14A685078117800022B4A084333
:10A35000801803280FD801F05BF802254439E06823
:10A3600001F0D6F8C0B20723B84204D37B19019399
:10A37000152B02DD0D231800FEBDE0682A00310018
:10A38000C01900F0B5FF6B4600209B88E268D054EE
:10A390001B4B1B68834203D01B68834200D0984745
:10A3A0000023E8E70B23002FE5D1022DE2D17378DB
:10A3B00032781B021343E2681380114B1B68002B99
:10A3C000EED01B68002BEBD00120E8E70B23002F19
:10A3D000D1D1062DCED12A003100E06800F088FFEF
:10A3E000DEE70B23002FC6D1012DC3D132787533A0
:10A3F000012AC0D8E3681A70D2E7C04600D6FFFF32
:10A400009069FF1F70B50C001500072837D800F0C1
:10A41000FFFF041436361B36242E182015290BD8BE
:10A42000184E16220021300000F03AFF22002900C9
:10A43000300000F05DFF002070BD18200229FBD124
:10A440001288114B1A80F6E718200829F4D10A0067
:10A450000E48290001F05CF9EDE718200129EBD145
:10A460000B4B10780B49DA69FFF7DEFEE3E71820A3
:10A470000129E1D1064B10780749DA6BF4E7022095
:10A48000DAE7C0467869FF1F2E45FF1F2445FF1FEE
:10A49000B444FF1FDC44FF1FFC44FF1F030010B542
:10A4A0000020DB0704D50721024A034800F08CF89E
:10A4B00010BDC046C4BA0011B444FF1F054A0300D2
:10A4C0001068002803D082889A4201D180687047C2
:10A4D0000068F6E7946BFF1F0A88030008009A42A1
:10A4E00004D08A8804309A4200D0002070470000CF
:10A4F000F8B5F82200230D4F0D4E79680500424350
:10A500003370994200D07B600A4C0021200000F09B
:10A51000C7FE00231A007C60AB4202D100203370DA
:10A52000F8BD01332280DBB2F834F5E7946CFF1FED
:10A53000906CFF1F986BFF1F73B56B460190060070
:10A54000684615001980FCF733FF041E11D1002D59
:10A550000FD07689002E11D00C2001F099F8002838
:10A560000ED0084A0460136886808560002B02D1F3
:10A570001060200076BD1A001B68F7E70224F8E798
:10A580001324F6E7946BFF1F012100220A4B10B53C
:10A5900049420A4C198099809A719A70084B207030
:10A5A000012019805A60FFF7A3FF2078FCF75EFFB7
:10A5B0000448FDF719FF10BD9869FF1F9C6CFF1F31
:10A5C000946CFF1F75A60011022310B5002802D05D
:10A5D000FFF7B2FF0300180010BD0000030010B524
:10A5E0000020DB0704D50421024A0348FFF7A4FF3B
:10A5F00010BDC046D8BA00113445FF1FF0B50E2675
:10A6000087B003930CAB1F8802ABF6180500080057
:10A6100031000292FDF74EF804000120002C0FD00B
:10A620003088FFF74BFF03000E20002B08D05E6838
:10A63000002E05D021002800039B029A0097B04706
:10A6400007B0F0BD0A4B10B5984207D10122002394
:10A6500052420A808B708A808B7110BDFFF73CFFDD
:10A660000028FAD001235B42038000238370F4E7C3
:10A67000FFFF0000F8B5050001290AD1134E0024A0
:10A680003388F827AB4219D028001149FFF7DAFFC9
:10A6900006E0022904D10139FDF724FF0028EDD09E
:10A6A000F8BD3B0063437268D018D35A002B09D021
:10A6B0003A00002100F0F4FD0134E4B2054B1B78B0
:10A6C000A342EED801235B423380DDE7946CFF1F89
:10A6D0009869FF1F906CFF1F10B5FFF7FDFE030088
:10A6E0000020834200D0987810BD0000F0B589B0FA
:10A6F0001C000EAB80CB03901E8810AB1B7804921D
:10A7000002930B7A0D00DB0616D42B780593022BEF
:10A7100024D00498FFF7D2FE002812D003689C468C
:10A72000002B0ED0029B2200019329003B006446BF
:10A7300003980096A04705E00498FFF7BFFE0028A5
:10A7400002D10E2009B0F0BD8368002BF9D00A2297
:10A750002900039898470028D7D0F3E76B6858780A
:10A760001A786B4B000210439842D2D8043B9842AF
:10A7700010D2684B984242D015D8674BC0180128B8
:10A78000C7D80B20002EDDD1EB681A7859683A80C3
:10A79000200028E0614BC018032800D979E000F0C0
:10A7A00037FE846A789E5E4B9842B2D10B20002E11
:10A7B000C8D101233B80EB6831001B782370688986
:10A7C000013080B2FCF776FF3A88031E0ED0017884
:10A7D00002328A183A80428962704289120AA27053
:10A7E00059680278E01C00F083FD06E004323A80EC
:10A7F00031000422601C00F053FD0020A2E70B2072
:10A80000002E9FD1EB6807A91E8804233B80330AE2
:10A81000300026706370FCF74DFF051E28D004AB96
:10A820009A890E2304A95B183E49C668FCF7B6FF57
:10A8300000280BD12B783C486A680599FBF76CFB24
:10A84000002803D1012304AA5B42D3813278022A73
:10A8500006D17168201D00F04BFD3B8802333B8020
:10A860000E2304AA9B181B88A3701B0AE370C4E77D
:10A8700004ABDE81F4E70B20002E00D062E7E9682C
:10A880000398FFF729FF02233B802070000A6070C5
:10A89000B3E70B20002E00D054E70222EB681B88A0
:10A8A0003A8023701B0A6370A7E7E86800F030FE67
:10A8B000C2B203000720B24200D243E70DD0029992
:10A8C000DBB27118994202DB921BD3B20293029B56
:10A8D000E9681A003B8089195AE70023F6E70B2044
:10A8E000002E00D02EE70722EB683A801A782270FB
:10A8F0005A7862705A88A2705A88120AE2701A79DD
:10A900002271DA886271DB881B0AA37175E7C04681
:10A91000042900000228000000D8FFFFFFD6FFFF37
:10A9200003280000FFFF000008BA0011F0B58DB049
:10A930006B460020089120229B5E83423DDAA64BA5
:10A94000187800F0DDFC071E32D00378B02B2CD134
:10A950000079023816281FD800F012FC17001E00DC
:10A960001E001E0031001E0096001E001D011E006C
:10A9700052011E0073011E00CD011E0050021E0078
:10A980001E001E008E021E00E302944B94491B8899
:10A9900078880B80FBF700F83800FCF781FF914BBB
:10A9A0001B68002B01D038009847380000F010FDDC
:10A9B0008020089B0002434018000DB0F0BDF62235
:10A9C0000021874800F06CFC0BAA3B7B7989388911
:10A9D00000923A000D32FCF785FD0400804B1B7895
:10A9E000002C3FD146E0804B788805937F4B410097
:10A9F000CB5A0BAE073BDBB23288029300230193A4
:10AA00007B4B210006930093059BFFF76FFE744D6F
:10AA1000002810D1069B3A8A1B889A420BD1380035
:10AA20000599123000F024FD002804D02B786289AB
:10AA30009B00EB185A80162306A81B1832882000AA
:10AA40007989FCF7ABFE2B7804009A00AA1851888C
:10AA50000029C3D00133DBB22B70002807D006A930
:10AA6000C98A9180634A12889A42BCD802E00121C7
:10AA700049429180002B04D059497888FAF7C0FFE9
:10AA80008AE73E890A2479E000253E89574B0693E0
:10AA90007B88069A5B009B5A033B9D4202DB002D9C
:10AAA000F0D05BE0162206A812183B7B7989009251
:10AAB0003A0030000D32FCF715FD0590002858D003
:10AAC0004689017A7888FCF7D7FC041E44D1464BAE
:10AAD00078880793069B4100C95A454B0439C9B28F
:10AAE00006AAD28A06930291019400930599079BC6
:10AAF000FFF7FCFD041E2FD1069B39491A88931CD1
:10AB0000002D26D14B807988384B4900CB5A5119FA
:10AB1000033B8B4220DD059B31485B8941190B715A
:10AB2000A91C0135C9B2EDB2059145191B0A2B715B
:10AB3000059B2D490433181800F0DAFB2C4B059ABD
:10AB40001B88D318DDB22C4B9E4205D00136B6B21D
:10AB50009CE749889942D6D0002D0CD0204C280083
:10AB6000618800F0FDFC207021007888FAF758FF1A
:10AB700012E7059CF0E7002C00D183E77B78142BCB
:10AB800000D109E716493B794E800B700C7178882B
:10AB9000FAF7F8FE00E7162406ABE418210038891E
:10ABA000FCF788FD011E00D1B7E1788822880F4CA0
:10ABB00045002C5B0A4D013CE4B2029400240F4B8B
:10ABC00001940095FFF792FD041E00D014E12900C6
:10ABD0007888FAF735FFDFE69C6CFF1F2044FF1FE3
:10ABE000A069FF1F9469FF1F9A6AFF1FD065FF1FAE
:10ABF000906BFF1F1E44FF1FFFFF0000A269FF1F95
:10AC0000162406ABE41821003889FCF753FD011E19
:10AC100000D182E178882288AE4C45002C5BAE4D95
:10AC2000013CE4B202947C89AC4B01940095FFF79F
:10AC30005DFD041E00D0DFE029007888FAF70AFFE6
:10AC4000AAE60025A44B1D803B00FE331B78A24AD8
:10AC500078880792AB4208D99E4B128806930699D2
:10AC600043005B5A013B9A4203DB0799FAF7FCFE6B
:10AC700092E616246B00FB18059306ABE418059BBF
:10AC800021001889FCF716FD011E03D1059B012444
:10AC90001E8973E77888924B2288069C09934300AB
:10ACA0001B5B904E013BDBB20293002300960193A5
:10ACB000099BFFF71BFD041E02D0059B1E895DE763
:10ACC0007B88069A5B009B5A079A10883288121874
:10ACD000934202DC1B1A013B33807F4C02303288E6
:10ACE0000999001900F004FB2388328801359B186C
:10ACF0002380EDB2A8E70BAA3B7B798938890092C3
:10AD00003A000D32FCF7EEFB00250590059B002B69
:10AD100004D10A24002D00D16EE060E0059B788804
:10AD2000197AFCF7A9FB0100041E63D1694C6C4B36
:10AD3000788806940993069B4400E45A694B063CC4
:10AD4000E4B20BAE32880793029401910093059907
:10AD5000099BFFF7CBFC041E4CD1079B5E491B8867
:10AD60001A1D002D30D14A80059B5B4C5A8963190E
:10AD70001A716B1C9BB2E318120A1A71162306A8EB
:10AD800032881B1879890598FCF708FDFF21AA1C59
:10AD90002E1D03350B00059092B2B6B2ADB200285D
:10ADA00003D006ABDB8AD9B21B0AA2186519117150
:10ADB0002B714C4D301D2A884949201800F098FA13
:10ADC0002B88F618B5B2A1E74988914207D17A8855
:10ADD00006995200525AEB18053A9A42C4DC3E4C8E
:10ADE0002800618800F064FA207021007888FAF762
:10ADF00045FED1E5002DF2D13E89BFE6162606AB11
:10AE0000F61831003889FCF755FC3D000400FF3589
:10AE100000282DD0037A9B060CD400227B89398927
:10AE2000788800923A000C32FFF7E8FB041E10D03D
:10AE30003E8915E03088FFF741FB00281AD083686F
:10AE4000002B17D02100122278889847041EE4D0E6
:10AE5000EEE7AB78002B02D17888FAF71FFE0026C8
:10AE6000AB78002B00D097E5002C00D194E585E667
:10AE70000124DDE70E24DBE7162506ABED182900DB
:10AE80003889FCF717FC041E47D0037A9B0611D4BF
:10AE9000154A7B881188994203D01448814207D112
:10AEA0001380134BF8261D780023D9B2A94221D371
:10AEB0000924A1E72888FFF701FB00282FD0836829
:10AEC000002B2CD02100122278889847041EDFD056
:10AED00092E7C046D065FF1FA069FF1FA269FF1F50
:10AEE0009A6AFF1F906BFF1F946CFF1FFFFF00000B
:10AEF000906CFF1F31005943546801336018615A48
:10AF00000029D2D13C0008342100F82200F0F0F9E9
:10AF100021007888FAF7CAFD3EE501246CE70E248B
:10AF20006AE71D4B1A887B889A4231D07888FAF7F5
:10AF3000C7FD31E5F823059851684343CD18C95A38
:10AF400000291FD03B7A012B0BD16C88AB88788805
:10AF5000AA1D0094FFF752FB041E02D000233B728F
:10AF60002E88F8220021280000F09AF900232B8077
:10AF7000059B0133DBB20593084B05991B78064A04
:10AF80008B42D7D801235B421380002CCED0F5E54D
:10AF9000002634000596EFE7946CFF1F906CFF1FAE
:10AFA00070B504000E001500FFF796FA031E08D1D5
:10AFB00031000548FFF790FA03001120002B02D062
:10AFC0001C8000209D7070BDFFFF0000F8B50B4F86
:10AFD00006003B780D001400FF2B0ED00A2000F075
:10AFE000DFF8011E09D0B1230380002346800371DE
:10AFF000C5800481387800F0B3FBF8BD7545FF1FAC
:10B00000F7B50F0008A90600088809A90B240988CC
:10B01000002821D10234022B1ED1557813782D023D
:10B020001D432B008B4301937334002B14D1FB6819
:10B03000300019000093FFF74FFB019C85420BD0B5
:10B040002A0030000099FFF7ABFF041E04D12A004C
:10B0500030007989FFF7BAFF2000FEBDF0B50E7809
:10B0600085B003900AA805880120022E0DD14C68F6
:10B070002778647824023C43054FBC4205D10398ED
:10B08000DBB201960095FFF7BBFF05B0F0BDC046EF
:10B090000229000010B504000C4800F021FA0C4809
:10B0A000A16B00F01DFA0B48E16B00F019FA0A4899
:10B0B000216C00F015FA094B0948196800F010FAE4
:10B0C000084B1B68002B00D09847FEE7DAB8001148
:10B0D000F0B80011FFB800110EB9001104ED00E046
:10B0E0001DB90011A06CFF1F002307B501A8019333
:10B0F000FFF7D0FF044A0548002110B5121A00F0EE
:10B10000CFF8F8F759FCFEE7A46CFF1F7845FF1F46
:10B1100001B40248844601BC604700BFC926000054
:10B1200001B40248844601BC604700BF093BFF1FD1
:10B1300001B40248844601BC604700BFF94C0100DD
:10B1400001B40248844601BC604700BF213AFF1F9A
:10B1500001B40248844601BC604700BF0D520100A3
:10B1600001B40248844601BC604700BFE1170000FB
:10B1700001B40248844601BC604700BF5549010044
:10B1800001B40248844601BC604700BF593CFF1F20
:10B1900001B40248844601BC604700BF75A90000A5
:10B1A00001B40248844601BC604700BF1D4D010048
:10B1B00001B40248844601BC604700BFE548000076
:10B1C00001B40248844601BC604700BFD91B00009F
:10B1D00001B40248844601BC604700BF9938FF1F94
:10B1E00001B40248844601BC604700BF4134FF1FE0
:10B1F00001B40248844601BC604700BF8D3AFF1F7E
:10B2000001B40248844601BC604700BF45510100BB
:10B2100001B40248844601BC604700BF9135FF1F5E
:10B2200001B40248844601BC604700BFC94A01001E
:10B2300001B40248844601BC604700BFB54C010020
:10B2400001B40248844601BC604700BF2951010097
:10B2500001B40248844601BC604700BF0134FF1FAF
:10B2600001B40248844601BC604700BF1147010099
:10B2700001B40248844601BC604700BFEDA5000050
:10B2800001B40248844601BC604700BFED4A01009A
:10B2900001B40248844601BC604700BF0189000038
:10B2A00001B40248844601BC604700BF154D01004F
:10B2B00001B40248844601BC604700BF090E00008B
:10B2C00001B40248844601BC604700BFC51D0000B0
:10B2D00001B40248844601BC604700BF4D1F000016
:10B2E00001B40248844601BC604700BF7D18FF1FBF
:10B2F00001B40248844601BC604700BFE94C01002C
:10B3000001B40248844601BC604700BFF54E01000D
:10B3100001B40248844601BC604700BFA134FF1F4E
:10B3200001B40248844601BC604700BF21240000EC
:10B3300001B40248844601BC604700BFD9490100FE
:10B3400001B40248844601BC604700BFC95C0100EB
:10B3500001B40248844601BC604700BF017F000081
:10B3600001B40248844601BC604700BF9DA90000AB
:10B3700001B40248844601BC604700BF055E00007E
:10B3800001B40248844601BC604700BF5147010038
:10B3900001B40248844601BC604700BFE9280000B0
:10B3A00001B40248844601BC604700BF3555000027
:10B3B00001B40248844601BC604700BFC53F00009D
:10B3C00001B40248844601BC604700BF6939FF1FD1
:10B3D00001B40248844601BC604700BF434D0100F0
:10B3E00001B40248844601BC604700BFE537FF1F37
:10B3F00001B40248844601BC604700BF014C010013
:10B4000001B40248844601BC604700BF1D4B0100E7
:10B4100001B40248844601BC604700BF453CFF1FA1
:10B4200001B40248844601BC604700BF8552010058
:10B4300001B40248844601BC604700BFD1A50000AA
:10B4400001B40248844601BC604700BF691F000088
:10B4500001B40248844601BC604700BF5118FF1F79
:10B4600001B40248844601BC604700BF8D12000051
:10B4700001B40248844601BC604700BFCD4C0100C6
:10B4800001B40248844601BC604700BF2526000085
:10B4900001B40248844601BC604700BF3D1800006B
:10B4A00001B40248844601BC604700BFE139FF1F78
:10B4B00001B40248844601BC604700BF8B520100C2
:10B4C00001B40248844601BC604700BFC5210000AA
:10B4D00001B40248844601BC604700BF353BFF1FF2
:10B4E00001B40248844601BC604700BFE53A010050
:10B4F00001B40248844601BC604700BF012400003B
:10B5000001B40248844601BC604700BF9130FF1F70
:10B5100001B40248844601BC604700BFDD5201000F
:10B5200001B40248844601BC604700BF151BFF1FE1
:10B5300001B40248844601BC604700BF55220000A8
:10B5400001B40248844601BC604700BFB14E000010
:10B5500001B40248844601BC604700BFDD30FF1FD4
:10B5600001B40248844601BC604700BF350E0000AC
:10B5700001B40248844601BC604700BF6932FF1F26
:10B5800001B40248844601BC604700BFA139FF1FD7
:10B5900001B40248844601BC604700BF851F00001B
:10B5A00001B40248844601BC604700BF291C00006A
:10B5B00001B40248844601BC604700BF456B0100EE
:10B5C00001B40248844601BC604700BF5539FF1FE3
:10B5D00001B40248844601BC604700BFB70E0000BA
:10B5E00001B40248844601BC604700BFB352010069
:10B5F00001B40248844601BC604700BF056A0000F0
:10B6000001B40248844601BC604700BFC9A90000DC
:10B6100001B40248844601BC604700BFC56D01000B
:10B6200001B40248844601BC604700BF311B0000E2
:10B6300001B40248844601BC604700BF5952010072
:10B6400001B40248844601BC604700BF6DBC0000E5
:10B6500001B40248844601BC604700BF091B0000DA
:10B6600001B40248844601BC604700BF313CFF1F63
:10B6700001B40248844601BC604700BF6571010007
:10B6800001B40248844601BC604700BFADAE000073
:10B6900001B40248844601BC604700BF3D4B010035
:10B6A00001B40248844601BC604700BF2146010046
:10B6B00001B40248844601BC604700BFF30E00009D
:10B6C00001B40248844601BC604700BF1537FF1F24
:10B6D00001B40248844601BC604700BF5D1700000A
:10B6E00001B40248844601BC604700BFC132FF1F5D
:10B6F00001B40248844601BC604700BF45500000C9
:10B7000001B40248844601BC604700BFA54F010058
:10B7100001B40248844601BC604700BF810E0000AE
:10B7200001B40248844601BC604700BF791800009C
:10B7300001B40248844601BC604700BF51250000A7
:10B7400001B40248844601BC604700BF0933FF1FB3
:10B7500001B40248844601BC604700BFA94601000D
:10B7600001B40248844601BC604700BF594F010044
:10B7700001B40248844601BC604700BF8132FF1F0C
:10B7800001B40248844601BC604700BF090E0000B6
:10B7900001B40248844601BC604700BFF136FF1F78
:10B7A0000002010302030303040305020602070269
:10B7B000080209000A030B030C020D020E030F031B
:10B7C000100311031303140315001600813D00112B
:10B7D000B53D00110000000002000000E2B70011BA
:10B7E000192A0F180A000000F1590000FD2400007A
:10B7F00041460100F17A0011059B0011596F0011BB
:10B80000F5780011ED5000112DA90011A14D001186
:10B81000793F0011A9400011000000001616000039
:10B82000020000002CB80011F4FFF3FFD2FC00006E
:10B830008D41001100000000000000005475796186
:10B840000056302E3700303030310067697468752B
:10B85000622E636F6D2F70767678004254483031D7
:10B86000000000000200000078B80011292A282AF0
:10B87000272A262A252A242A0A180000E204000082
:10B880007102000078EC00007440000010270000F6
:10B8900060F0000006640000204E00000000000080
:10B8A000000000001F501D00023C020000011400B7
:10B8B0000700000083020000303132333435363760
:10B8C0003839414243444546005048592B36325896
:10B8D00058504C555330353034005B486172642009
:10B8E0006661756C742068616E646C65725D0A00D7
:10B8F0004C522020203D203078253038780A0050E6
:10B90000432020203D203078253038780A005053DD
:10B910005220203D203078253038780A00494353A2
:10B9200052203D203078253038780A00FD5400112F
:10B9300051550011000000000200000044B9001140
:10B940006F2A6E2A1A18000001A0000000000000F3
:10B950006410B71DC8206E3BAC30D9269041DC7610
:10B96000F4516B6B5861B24D3C7105502083B8EDBA
:10B9700044930FF0E8A3D6D68CB361CBB0C2649BDE
:10B98000D4D2D38678E20AA01CF2BDBDFB349B5F03
:10B990008000008000100000000000005B5B0011D0
:10B9A000E57100117F5B0011ED750011035C001162
:10B9B000C3750011795C001199750011CB5C001101
:10B9C00061770011335D001161770011655D001131
:10B9D0001B770011795C001151750011F15C0011A9
:10B9E000F97600110000000000000000D75D001192
:10B9F000F9760011395E0011FD710011052A042A43
:10BA0000012A002A02290328012800280118001809
:10BA1000000000000000000000000000000000879F
:10BA200001010201020101020102030304010301F9
:10BA3000010101010303020103000D000E001000CB
:10BA4000110013001401070108010A010B011C0178
:10BA50001D02040205020702080219021A021C0252
:10BA60001D0301030203170002010005040008077B
:10BA7000000B0A001716001D1C010201010504013C
:10BA80000E0D011110011413011716011A190202EB
:10BA900001020B0A020E0D021110021413021716F6
:10BAA000030504030807030B0A030E0D000102033C
:10BAB00007090A0B0E0F101112141718191A1B1F61
:10BAC0002021220075A2001131A300110000000006
:10BAD000020000000EBA0011000000005DB000116D
:0CBAE00000000000020000000CBA001181
:020000041FFFDC
:1000000000000000DD3E0011E8B70011E4B7001168
:100010008462FF1F000000000000000000000000DC
:1000200000000000000000000000000000000000D0
:1000300000000000000000000000000000000000C0
:1000400000000000000000000000000000000000B0
:1000500000000000000000000000000000000000A0
:100060000000000000000000000000000000000090
:100070000000000000000000000000000000000080
:100080000000000000000000000000000000000070
:100090000000000000000000000000000000000060
:1000A0000000000000000000000000000000000050
:1000B0000000000000000000000000000000000040
:1000C0000000000000000000000000000000000030
:1000D0000000000000000000000000000000000020
:1000E0000000000000000000000000000000000010
:1000F0000000000000000000000000000000000000
:1001000000000000000000000000000000000000EF
:1001100000000000000000000000000000000000DF
:1001200000000000000000000000000000000000CF
:1001300000000000000000000000000000000000BF
:1001400000000000000000000000000000000000AF
:10015000000000000000000000000000000000009F
:10016000000000000000000000000000000000008F
:10017000000000000000000000000000000000007F
:10018000000000000000000000000000000000006F
:100190006534FF1F5533FF1FC166010000000000DA
:1001A000000000000000000000000000000000004F
:1001B000000000000000000000000000000000003F
:1001C000000000000000000000000000000000002F
:1001D000000000000000000000000000000000001F
:1001E000000000000000000000000000000000000F
:1001F00000000000000000000000000000000000FF
:1002000000000000000000000000000000000000EE
:1002100000000000000000000000000000000000DE
:1002200000000000000000000000000000000000CE
:1002300000000000000000000000000000000000BE
:1002400000000000000000000000000000000000AE
:10025000000000000000000000000000000000009E
:10026000000000000000000000000000000000008E
:10027000000000000000000000000000000000007E
:10028000000000000000000000000000000000006E
:10029000000000000000000000000000000000005E
:1002A000000000000000000000000000000000004E
:1002B000000000000000000000000000000000003E
:1002C000000000000000000000000000000000002E
:1002D000000000000000000000000000000000001E
:1002E000000000000000000000000000000000000E
:1002F00000000000000000000000000000000000FE
:1003000000000000000000000000000000000000ED
:1003100000000000000000000000000000000000DD
:1003200000000000000000000000000000000000CD
:1003300000000000000000000000000000000000BD
:1003400000000000000000000000000000000000AD
:10035000000000000000000000000000000000009D
:10036000000000000000000000000000000000008D
:10037000E9B00011000000000000000000000000D3
:10038000000000000000000000000000000000006D
:10039000000000000000000000000000000000005D
:1003A000000000000000000000000000951AFF1F80
:1003B000000000000000000000000000000000003D
:1003C000000000000000000000000000000000002D
:1003D000000000000000000000000000000000001D
:1003E000000000000000000000000000000000000D
:1003F00000000000000000000000000000000000FD
:08183800B070FF1F4118FF1FF3
:10184000024981F3088802F0C3FA0000B070FF1F5C
:1018500010B502F035FB072804D0122808D0022862
:1018600008D010BD044A0420136B01331363F8E75A
:101870000220F6E71420F4E77866FF1FF8B50700AA
:101880000C0026002500503630785135002804D150
:101890000300287058342370F8BD2978CA00481E08
:1018A0008141A3183800A25C5B68C9B2FFF7D0FF82
:1018B00000280DD12B78DA00A218013350602B706C
:1018C0003378044A013B3370136A01331362D8E75B
:1018D0000123DFE77866FF1F5C234343074910B508
:1018E000C9180B0058331B78012B05D1FFF7C6FF31
:1018F000034A936A0133936210BDC046AC66FF1F72
:101900007866FF1F10B502F043FA064A0121130062
:1019100010CB4942D967044B136002F029FC200028
:1019200010BDC04600E100E01000100010B504003A
:1019300002F02EFA024B1C6002F01AFC10BDC046E9
:1019400000E100E010B5040002F022FA4021094A4B
:10195000200013688B43136002F0A2F901F064FDCC
:101960000022054B01201A60044B04321A6002F079
:1019700057FAFEE71CF00040C4F00040C0F0004001
:10198000431E5A425341A022F0B5D2015B4213409C
:10199000154D164A40019B182A18127E8BB00191F2
:1019A000002A1BD01A000832D46F0022E6B206AF1C
:1019B000E4B294420EDC2818C369002B08D00199C8
:1019C00002AA117106AA049202AA167303A89847E4
:1019D0000BB0F0BD1978B9540132EAE71A7D1A78D4
:1019E00006AB01261A70E6E73869FF1F0040004089
:1019F000F0B5254B04004001C25C85B0002A2BD015
:101A00001A18117E002927D0917E002924D011793F
:101A1000022921D11689D788D168F51BADB22A1CBD
:101A2000102D00D9102292B2BE4217D118180123EE
:101A300003710023C269C38003819A4206D06846BD
:101A4000032103730171029301A890470820002C21
:101A500000D0192001F034FC05B0F0BD013C654216
:101A60006C41A0256442ED012C40084D1B186419FF
:101A7000074D0633013A92B2AA42EDD01888461CAF
:101A80001E80085C2070F5E73869FF1F00400040A9
:101A9000FFFF00000F220E4B10B59868104002386F
:101AA0000A280BD802F0CEF80D0A0B0A0A110A0A0E
:101AB0000A0A060002210020FFF762FF10BD012183
:101AC000F9E70020FFF794FFF8E7DB6FF6E7C04681
:101AD000004000400F220E4B10B5986810400238AD
:101AE0000A280BD802F0AEF80E0A0B0A0A120A0AEC
:101AF0000A0A060002210120FFF742FF10BD012162
:101B00000800F9E70120FFF773FFF7E7DB6FF5E760
:101B10000090004013B5334C2378072B3DD8324B4F
:101B20001A78324B002A39D18022196852020A43AE
:101B30001A60252001F034FF20232D4A11680B4341
:101B4000802113606B460422C905086807331042E0
:101B500028D080210422C905C86810422ED08021D7
:101B60002020C905CA688243CA6014221A701A78F4
:101B7000002A2FD18021C905C86820320243CA60DB
:101B800014221A701A78002A28D11A4B1A7D22784A
:101B90005A601D221A705932DA6013BD1A6816494C
:101BA0000A40C5E7086802430A6014221A701A78CE
:101BB000002ACED01A78013AD2B2F7E7C8680243B9
:101BC000CA6014221A7019784A1ED2B21A700029FB
:101BD000F9D1C4E71A78013AD2B2C7E71A78013AC4
:101BE000D2B2CEE7B044FF1F7845FF1F3CF0004063
:101BF000A844FF1F00200040FFFFFEFF564B70B5BA
:101C00001B68012B03D1554A936D0133936502F094
:101C100067F8534B534A1860534B544C1A600123D6
:101C2000534A1360534A13602378002B06D00622D0
:101C30005149524802F0DCF900232370504A514BBD
:101C400010681B78C1B2002B0ED14F4CC0B2237864
:101C50005BB2002B4FDB237824785BB264B21B04A9
:101C600024021B191B1813600B1C50294ED950233A
:101C7000464A47491078DBB2FF2202284BD1086858
:101C8000444C454D267890432A78964254D9227880
:101C900024782E78023B5D10A31B6B435201D31AAC
:101CA00010335B111843086002F032F9031F012B57
:101CB00045D83A4B1B78002B06D0394B1B78002BAC
:101CC00002D0002002F034FAA122364B920099781B
:101CD000354B4A431B689B18832292009B181B7844
:101CE000033B012B03D8AF20400002F0D9F80122BA
:101CF0002E4BDA8270BD237824785BB264B2FF3356
:101D0000FF341B0424021B190138ABE7CAB2022AB4
:101D1000AED20223ACE70868254C264D26789043C6
:101D20002A78964208D9227824782D78023B5B10D5
:101D3000641B63435201B2E72378DBB2B2E70228A7
:101D4000D5D11D4B1B78013B022B03D91B4B1B78B4
:101D5000022BCCD16C20C8E79809FF1FFC0FFF1F96
:101D6000B065FF1FFF3F000014100340B465FF1F64
:101D70000C10034000100340D50BFF1F7211FF1F12
:101D8000B40003408C09FF1F680AFF1F490AFF1FA8
:101D900094000340460AFF1F470AFF1FF908FF1F70
:101DA0002209FF1F300DFF1F3409FF1FBC0BFF1F4F
:101DB000440AFF1F450AFF1F1C09FF1F2309FF1FBD
:101DC00010B502F0C5F80022014B1A8010BDC046C4
:101DD000AC65FF1F10B502F05BF8A121054A890030
:101DE0009478054A61431268044B5218528C1A8049
:101DF00010BDC046300DFF1F3409FF1FAC65FF1F2B
:101E000010B50D4B0D4A9978A1239B004B431268E6
:101E1000D218531DD97F0A4B1B88994209D2441C02
:101E200007D0C82805D0D2695B1A5A43054B5343E3
:101E3000C01802F065F810BD300DFF1F3409FF1FF8
:101E4000AC65FF1F7102000070B5244D2B68002B9C
:101E500028D001F0C5FF2B68D8402B680400002B68
:101E600027D001F04DFF2B68D8401D4B1D4A9978B3
:101E7000A1239B004B431268D118D25C91239B0095
:101E8000002A20D0CA580132CA50174B17491B6884
:101E90000868834214D3D23B181A012A1AD0144B73
:101EA000186070BD01F09CFF124B196802F0E8F851
:101EB000D3E701F025FF0F4B196802F0E1F8D4E7F2
:101EC0000D495B18E8E7CA500C4B1B68DB68E41847
:101ED000201AE4E7F530FF30E1E7C0461C08FF1F99
:101EE000300DFF1F3409FF1F9C09FF1FB065FF1F46
:101EF000A009FF1F1808FF1F2DFF3F00B865FF1F37
:101F000070B504000D00282916D10300A433C2883F
:101F10001B889B1A0B4A9BB293420DD906006A3666
:101F200005223100653001F0A3FE002804D1310004
:101F3000200002F01DF870BD2900200001F000FF14
:101F4000F9E7C046FE7F0000F8B50400012001F06B
:101F500007FF02F0D5F8174A174910600968030017
:101F60001648174E01601748776805680020AF4291
:101F700001D27068281A144D091928601348C162EB
:101F8000A421446A49032143416211490978002987
:101F900005D010490978022902D10F3B1360F8BD22
:101FA000012901D1083BF9E7032901D1053BF5E7F8
:101FB000033BF3E7E408FF1F28F00040340AFF1F4B
:101FC00028100040180AFF1F1C0AFF1F00F00040E5
:101FD0001C09FF1F4A0AFF1F70B580241025E40565
:101FE000A3682B43A36001F0ABFFA368AB43A360DE
:101FF00070BD0000F7B5160080221C001023D2052A
:102000000191916805000B43936000225A4BD73031
:102010001A6001F04DFE9D232A002F009B00EB5813
:10202000CA3201210092FC37002B01D00021009A16
:10203000386801F01DFF2900009BCB311A784F4B07
:10204000D3351A604B780A781B0213438A7812043E
:102050001A43CB781B061343494A1BBA13604B79CA
:102060000A791B0213438A7912041A43CB7931008F
:102070001B061343434A1BBA13606B782A781B0272
:102080001343AA7812041A43EB781B0613433E4A03
:102090001BBA1360019A330213433C4A13603C4B52
:1020A00022001B1B9C4603293DDCB3089A00130049
:1020B0005142B21A032A46D1354AE018511A8278A1
:1020C0004078120400020243E05C043302430A60D9
:1020D0000022FF2B4BDDF0222E4B12011A600F2243
:1020E0002D4B1A602D4A1368002BFCD00023224A86
:1020F00027491360091B321D0B191B68043A180A83
:1021000023706070180C1B0EA070E3700434002A5A
:10211000F2DC802210213B68D20501333B609368DA
:102120008B439360F7BD6346D578981893782D0656
:102130001B042B43157804392B43557804322D02A8
:102140002B430360AFE7022A0AD1114AE05C511A1F
:10215000E2185278120202430A6004339BB2B7E7D6
:10216000012AB5D10A4A521AE15C1160F5E7084923
:1021700059180A600433ACE7000004403C000440F6
:102180003800044034000440300004400C00044097
:102190000001044004000440100004401400044006
:1021A000F7B5150080221C001023D205009191681C
:1021B00007000B4393600023654AD730136001F09A
:1021C00077FD9D233E009B00F9583B00CA36320044
:1021D000FC33002900D07FE0586801F049FE390047
:1021E00032785C4BCB311A604B780A781B02134370
:1021F0008A78AC4612041A43CB78281D1B06134379
:10220000554A1BBA13604B790A791B0213438A792A
:1022100012041A43CB791B061343504A1BBA1360AE
:102220004B7A0A7A1B0213438A7A12041A43CB7A36
:1022300021001B0613434A4A1BBA1360009A2B0263
:102240001343484A13602200474B1B1B0093009B1B
:10225000CE785B1801938B7836061B0433430E78D7
:10226000043833434E78043136023343019E3360E1
:102270000328ECDC0321A808431C9B0029408000B4
:1022800003292BD13849E5185E18A9786D78E35CED
:1022900009042D022943194331600300083300214A
:1022A000FF2B2DDD314B324919600F21314B196065
:1022B000012327490B60304B19680029FCD0062107
:1022C0001B680B40042B20D080220020D20593688D
:1022D0000A318B439360FEBD01217DE7022908D1BD
:1022E00021495D18E1184978E35C09021943296026
:1022F000D3E70129D3D11C495918E35C0B60CCE723
:102300001948181801600433CAE7002310490B600C
:102310006346002B0CDC3B00FC335A681021013271
:102320005A608022D205936801208B439360D2E7E4
:10233000009B9B181B68190A13705170190C1B0E17
:10234000D37004235B4291709C440432E0E7C046A2
:10235000000004403C0004403800044034000440C5
:10236000300004400C00044000010440040004401C
:10237000080F0000100004401400044070B5061E51
:1023800019D00222614B9B799343012B13D1604BEF
:102390001A78FF2A0FD15A78FF2A0CD19A78FF2A8F
:1023A00009D1DA78FF2A06D11A79FF2A03D15B799D
:1023B000FF2B00D1A7E0574B0C201A78012A08D038
:1023C0000022554D1A702B781A00093A042A01D8B8
:1023D000212070BD5A1F012AFAD94C4CA07B042839
:1023E00000D990E0A279032A00D98CE0821E012A4C
:1023F00003D862881F2A00D885E0002E61D0012E04
:1024000000D080E0A288012AE2D0002B0AD1013856
:10241000032803D801F016FC151D19151F202E7076
:1024200001F0B6FD2B785A1E032A16D800253B4B27
:102430001D602823237501F0C3FCA8422ED0A5807F
:10244000C6E7022320202B70EAE7042322202B700A
:10245000E6E7032321202B70E2E7073B012BB7D8E7
:102460002F4B1B68DB6A9B06B2D52E4B1A78002ACD
:10247000AED1A27B911E012901D9002AA8D1022246
:1024800080211A702823284D89012878237501F0AE
:1024900047FD80212878890101F0D2FD0123A38026
:1024A000224B1B78002B0AD0FA228021204B92006D
:1024B0001B8809025A431C4B187801F0C9FC002004
:1024C00087E701F065FC2B78A680073B012B06D936
:1024D00018482E7001F0DCFD1E2001F059FD114B53
:1024E000114C1A78002A06D0802100222078890118
:1024F0001A7001F015FD01F03BFE802120780902E1
:1025000001F00EFDDBE7122063E7C046A60BFF1FBC
:102510006B09FF1F1A09FF1F1C09FF1F4809FF1F36
:10252000B865FF1F2309FF1F1B09FF1F2109FF1F9C
:102530002C09FF1F0010004010B5002901D001F048
:102540006FFD10BDF7B5604B01919978A1239B00F9
:102550004B435E4A060014681022E418D6235B0041
:10256000E0583623FF33E35C00279343222B41D10D
:10257000574B0F3A1A600760012501F0A9FD019B36
:102580001880E8235B00E35C002B01D0B34258DDE8
:102590000023504FFB70AD33FF33E3581A68002A15
:1025A00003D09B88DB439B071DD03823FF33E35CBC
:1025B000002B18D09B235B00E35C002B13D1D1339D
:1025C000FF33E35CB3420EDAA4235B00E15AE01868
:1025D000090A023101F03CFD23000122FE33013ED5
:1025E00001351A87FA70E8235B00E35C002B2AD0E0
:1025F000A8B2FEBD03683D00002BBED08188043028
:10260000090A023101F024FDD6235B00E3581F6064
:10261000B2E72300B133BA00FF33985801378188FD
:102620000430090A023101F013FDE8235B00E35C8A
:10263000BB42EEDCE822F61AED1800235200A35448
:10264000A6E70027F1E7200001F06AFB00281FD071
:10265000002E1DDD7319882647190193B60020004E
:1026600001F09EFD5A3080002018406801358188B5
:102670000430090A023101F0EBFC200001F0F8FC03
:10268000A3590133A351BD4202D0019B9D42E6D123
:10269000114BE35C002BABD095239B00E35C002B3C
:1026A000A6D00E4BE15A0029A2D00D4AA35C994254
:1026B00002D90133A3549BE700231A212000A3541D
:1026C00001F04EFD94E7C046300DFF1F3409FF1F97
:1026D00000140340E010FF1F5A02000072020000C5
:1026E0005E020000F8B51D4B1D4F1A78002A10D16C
:1026F000BA7B002A02D101321A7003E0032AFAD011
:10270000022AF8D001F05CFB00220120154B1A7060
:10271000F8BD154B154D1C68154B9E7801232B7089
:102720002878C0B200F0DEFCBB7B002B0BD101F09F
:102730006FFBA1239B007343E41883239B00E418E1
:1027400023782B70E4E7032B02D101F059FCF0E76A
:102750000020022BDCD101F013FBEAE71C09FF1F6C
:10276000A60BFF1F2309FF1F3409FF1F490AFF1F84
:10277000300DFF1FF0B587B00EAD2F780FAD2D785F
:102780000593AC46634614000E4D0CAA12782E78C1
:1027900003930D9B009201932200059B029701F089
:1027A0000FFC2E70012C01D0042C08D18022064988
:1027B0008B889343054A1278D20113438B8007B06C
:1027C000F0BDC0461C09FF1F6C11FF1F7809FF1FD9
:1027D0000B001B3B70B504003020E02B0DD813001C
:1027E000E025493BFF3B9BB2ED00AB4205D8034BD4
:1027F000200019825A8201F00BFC70BD8410FF1F6B
:1028000010B501F06DFA054B00205B68052B04D96B
:10281000034A5268D20200D4980810BD001000404C
:10282000FCE100E070B501F0B3FA0D4B1B68FC331E
:10283000DC691D6AFFF7E4FF6419844204D2094B86
:1028400001241B68002B07D004220024064B1A70B9
:10285000064A93690133936101F08AFC200070BD40
:10286000B865FF1F9809FF1F2309FF1FFC0FFF1FFB
:1028700070B50C4D2B68FC335C6A01F089FAFFF7E8
:10288000BFFF2B680025FC339B6AE318834204D208
:10289000054B1B68AB4200D1051B01F069FC280009
:1028A00070BDC046B865FF1F9809FF1FD722044BB3
:1028B00092009B5810B5002B00D0984710BDC04621
:1028C0000000FF1FF0B587B001F046F9FFF7EEFFFB
:1028D000CA4BCB4C04931B78022B45D1C94B1B68C8
:1028E000186A01F03DFAC84BC84A1A60C84BC94A79
:1028F0001A60A022C84B52001A60049B187801F09D
:10290000EFFAC649C64801F04BFAC649C64801F07D
:1029100047FA1022C54BFF201A60802252031A602A
:10292000802292031A60802212041A6001F000FCD7
:10293000012001F0ADF9FA20400001F0B1FB582070
:1029400001F0AEFABA4801F023FC012001F070FB5F
:10295000072001F0E5FB2268B64B1A4084235B0098
:102960001343236007B0F0BD01F042FAB24E02906B
:10297000322001F0F5F933681B0629D43C2001F020
:10298000EFF90F2001F0ECF99C4B1B78012B00D1E3
:102990001EE180223368A94D134200D0A7E02B68C6
:1029A000032013432B6001F0DBF901F021FA029BB5
:1029B0000299C31A5A1E814200D81A00A04B1A600D
:1029C000904B19681E2353439E4A9B18CB618AE79C
:1029D00001F00EFA80239C4ADB02116803900B433E
:1029E00013602268934B994F1A40282313432360A6
:1029F000032001F0B5F903203D6801F0B1F93B680F
:102A00000320DB03DB0B009301F0AAF93B68ED0325
:102A1000DB03ED0BDB0B8E4A0193AB18C22B30D8D6
:102A2000009B9B18C22B2CD8019B9B18C22B28D82B
:102A3000009B2A009D4200D21A00009B9D4200D9B3
:102A40001D00019B934200D21300019A954200D9C8
:102A500015005B1B122B14D80C22336814209343EF
:102A6000336033687B4A1340336001F079F9082101
:102A70003B682268DB038A432260774ADB0B1360E2
:102A80007FE7032001F06CF93B68DB03DB0B059368
:102A900001F0AEF9039B0399C21A531E814200D87C
:102AA00013006E4A93421BD9FF23356869492D0AEA
:102AB0001D4032686B1C1B060A401B0C134333601D
:102AC0000C23326800209A43083B1343336001F023
:102AD0004FF96348634BA840984206DCFEF732FF8B
:102AE000019B009D0093059B95E75F48F6E7002357
:102AF0005E4F554A3B6080231168DB020B43136035
:102B000080222B68032013432B6001F029F93B68D6
:102B1000052601333B6080232A685B0213432B6048
:102B20002268444B03201A40514B1343236001F0A9
:102B300017F90821454B1A682368D2038B43236099
:102B4000454B023900931B68D20B4B439A420CD879
:102B50009B1A3B2B0BD8236846490B4023602B68FC
:102B60000B402B60444B1A601FE7D31AF1E7013E7C
:102B7000F6B2002ED4D123683E4A134023602B685E
:102B800013402B603B68042B07D9BFF34F8F3B4B9F
:102B90003B4ADA60BFF34F8FFEE780222B680320A9
:102BA00093432B6001F0DCF82268224B03201A408B
:102BB00028231343236001F0D3F8244B009A1B68A9
:102BC000DB03DB0B1360082223689343236097E742
:102BD00007222C4D2B681340012B02D1002001F05D
:102BE0007FF9AB68284A02201340AB6001F0B8F8C7
:102BF0008023AA685B001343AB60D6E64A0AFF1F36
:102C00005CF00040B865FF1F000003400180063DF6
:102C1000BC00034034080000A4000340710200001F
:102C200014100040FFFF3F002810004000E100E0CA
:102C30003075000000FEFEFFC4F0004044F000408C
:102C4000A065FF1F7206000040F0004064F00040E5
:102C500091FCFFFFFF00FFFFA865FF1FE30C0000D2
:102C6000E88000005F361E0060361E001444FF1F1F
:102C700028000100FFFFFEFFA465FF1F00ED00E03C
:102C80000400FA053CF00040FFFEFFFF694E336888
:102C900088331B6883F3088801F09AF900F0C4FBBD
:102CA000654B664A1B68934207D0002001F060F82C
:102CB0000221634A13688B431360FFF703FE614BE5
:102CC000614C1878C0B201F013F90023A3600233FD
:102CD000A3605E4B0120236001F042F80323A36050
:102CE00001F086F8040000F0FBFF050001F080F819
:102CF000574B186001F024FA564B1968621A531E9C
:102D0000A14200D213008022D203934201D39B023E
:102D10009B0A3268D16AC90700D478E04E491C0C7E
:102D200009689BB24C4359432402090A64180327DB
:102D30004A49FC3293680A6849489B1A494A4A4EF4
:102D400012684A499B18414A34609A183B400193E3
:102D5000036892089C46019B0A6063440360042B4D
:102D600003D901323B400A6003600B684049E41814
:102D7000200001F085F93F4F3D493B68C3183B6097
:102D80002000019301F0FCF83B4C206808183849FA
:102D90002060884205D9019B01333B6001F0F0F8C7
:102DA000216000F08DFF354B1B78002B0ED000F01A
:102DB00097FF3168324B4A1B1B6812189A4233D274
:102DC000591A4919091A2F4800F0EAFF2E4C237AA4
:102DD000002B0FD000F084FF3168E3684A1B121803
:102DE000934224D9591A4919091A284800F0D8FFE2
:102DF00000232372264B83F3088801F059F8022040
:102E000001F0C6F8002000F0B3FF01F069F9DC0121
:102E100099000234641A5900641A09214B43803323
:102E2000CB40A408E41882E7FA218900CBE71949CE
:102E3000DBE7C046B865FF1F0C0AFF1FB641210340
:102E400010000040490AFF1F14100040C409000090
:102E5000100AFF1F340AFF1F380AFF1F200AFF1F36
:102E6000280AFF1F1C0AFF1F9C65FF1F240AFF1F63
:102E7000710200006008FF1F2C0AFF1F1C09FF1FC2
:102E8000E408FF1F00100040740BFF1F3C100040BF
:102E900000000020DC050000A022054B92009B589A
:102EA00010B5002B01D0984710BD01F059F8FBE791
:102EB0000000FF1FA122054B92009B5810B5002B6C
:102EC00001D0984710BD01F04BF8FBE70000FF1F51
:102ED000A222054B92009B5810B5002B01D09847B9
:102EE00010BD01F03DF8FBE70000FF1FA322054BDA
:102EF00092009B5810B5002B01D0984710BD01F0EF
:102F00002FF8FBE70000FF1FA422054B92009B58FF
:102F100010B5002B01D0984710BD01F021F8FBE758
:102F20000000FF1F70B500F0DBFE514B186004205D
:102F300001F02EF801F054F80400C30702D400F0A9
:102F40009FFE70BD00224B4B1A604B4B1878013826
:102F500004282CD800F076FE03231B1F2700200036
:102F600001F0D6F80128ECD0444C2378042B71D121
:102F700000F0AEFE002806D001F09AF8582000F0CC
:102F80008FFF02232370032001F002F8D9E720000D
:102F900001F096F8E6E7200000F0BAFEE2E7200034
:102FA00000F0A6FEDEE7200001F05AF8DAE700F0B4
:102FB000AFFF0500012808D1314B1B78053B012BE1
:102FC00003D82000FFF768FFCEE72C4B1B78022BBD
:102FD00001D0052B20D1022D28D12A4B9B7BAB435E
:102FE0001CD12000FFF766FF254B18780128BBD1C4
:102FF0006405B9D4234925224B7B034205D1233AEA
:1030000013405A42534126331A000B7D9342ABD9E9
:10301000322000F09DFEA7E7022D07D1184B1B7848
:10302000052B11D12000FFF753FFDDE7012D0BD158
:10303000012B03D12000FFF759FF95E7062B03D1A1
:103040002000FFF761FF8FE7200000F089FF022DCD
:103050008AD1C9E7032B04D10B4B987C00F000FF09
:1030600091E7072B8FD1094B987B00F0E1FE8AE7AF
:103070009C09FF1F9809FF1F9009FF1F2309FF1FCD
:103080001C09FF1FA60BFF1FBC0BFF1FD40BFF1F4C
:10309000FA210A4B0A4A49001A640A4A5A500A4A53
:1030A00004395A50094A08319A64094A5A50094A5F
:1030B0005C315A50084ADA667047C0460000FF1F6C
:1030C0007527FF1F7128FF1F2528FF1F7D23FF1F66
:1030D000E526FF1F011EFF1FD51DFF1F10B500F0C5
:1030E00099FD10BD8023F7B59C46264B264F0193D2
:1030F0002649274A274D284C284B02281AD16046DA
:1031000038600868264E3040802636033043086019
:1031100001990978002909D11660224A2A60224AB9
:103120002260E02219689143A03A1BE08021C90285
:103130001160F2E766463E600F68194E3E408027F8
:10314000FF023E430E600199097800290DD11760F6
:1031500001280ED1154A2A60154A2260E02219681A
:103160009143C03A0A431A60F7BD80218902116079
:10317000EEE7E0210F4A02432A600F4A22601A68F4
:103180008A43F0E74B0AFF1FE0000340D8000340EA
:103190009000034000000340500003404000034003
:1031A000FFFFE3FF0280063D804508220180063DC7
:1031B000806608220080069880550822F8B51E4BCC
:1031C00080261A68002014003440324232D11A6836
:1031D0001A4F32431A6001223B68063093433B602A
:1031E00000F0BEFD0122164D2B681E432E603B6889
:1031F0000A2613433B608027BF00124B1B683B42EB
:1032000011D1013EF6B2FF2E09D17E220E4B1C6871
:103210002B68E40B1440934323432B6005E0082004
:1032200000F09EFDE9E7002EEFD180222B686008B8
:1032300093432B60F8BDC046C4F000405CF00040F2
:1032400018F0004068F0004060F0004010B500F059
:1032500097FF01215820034A00F03AFEFFF7AEFF26
:1032600010BDC046600AFF1F10B578220021034838
:1032700000F09EFD00F0E4FD002010BDC068FF1FBF
:1032800070B5040000F084FD00230C200B4A0100FF
:1032900059438D18515C00290DD0A14208D101235A
:1032A00000246B7000F024FF00F062FF200070BD6E
:1032B00001330A2BEBD11224F6E7C046C068FF1F8A
:1032C00070B5040000F064FD002319001D000D4AD4
:1032D0001078002806D0A0420CD1557001310C3274
:1032E0000A29F5D1002B0AD100F0AAFD00F040FF19
:1032F000002070BD5078461EB0411B18EEE700F06C
:10330000F7FEF3E7C068FF1FF7B504000C200023A9
:1033100084460E4D019267465F43E85D7E19A042E8
:1033200012D000280BD10A4B9C4662461B7808330A
:103330001370019B70707C557160B360FEBD0133EA
:103340000A2BE8D10320F9E70720F7E7C068FF1F41
:10335000BC68FF1F8021204BC9051B6870B58B60BE
:103360001E4BC1241A680123FF2013434B611C4BE1
:10337000A4001A681B4B00251A601B4B1A681B4BD4
:103380001A601B4B1A5982431A51C52292009C584D
:103390008443BF38204398509C58164804408020EE
:1033A000C001204398509858134C0002000A014372
:1033B0009950124B1B78DB08AB4201DC002070BD3A
:1033C0002378002B06D0A368002B00D09847013546
:1033D0000C34EEE71220F2E7AC44FF1FA844FF1FB5
:1033E000B0F00040B868FF1FB4F00040B468FF1FA1
:1033F00000E100E0FF00FFFFC068FF1FBC68FF1F87
:10340000030010B51F2809D8072200201340072405
:1034100004490A78A24313430B7010BD0023062011
:10342000F5E7C046BC68FF1F034A04491368002043
:103430000B4013607047C0461CF00040FFFFC1FF07
:10344000054B06491B780A6805485B0702401B0BC1
:10345000134300200B607047BC68FF1F1CF0004046
:10346000FFFFC1FF70B50C25FFF7EAFF0A4B1C7880
:103470000A4BE4086543ED18002C01D1200070BD13
:103480002B78002B06D06B68002B00D09847013CAE
:103490000C3DF1E71220F2E7BC68FF1FB468FF1F84
:1034A00007B50422074801A900F034F9019B013354
:1034B00005D18023044ADB0411680B43136000200C
:1034C0000EBDC0461C18001114F00040F0B50500F8
:1034D0002026184B87B00493049B002B03D11124A2
:1034E000200007B0F0BD002102220B0001910091E5
:1034F000052000F05DFE02230F490A681A42FCD144
:103500000596059C631E0593002CFAD10B4A13689F
:10351000002BFCDA0F276F440121380000F040FD3A
:103520003B782B42DCD0052000F01AFC049B013BC9
:103530000493D1E7FFFFFF0790C8004000C8004098
:1035400007B500F025FC80220821D205936A01917D
:10355000002B01D10739916202210C4A11600199B7
:10356000481E01900029FAD1033111600531019103
:103570000199481E01900029FAD11160002B02D157
:103580008022D205936200F0F3FD07BD00C0004029
:10359000F0B52D4C89B02378002B4FD1FEF7B2F94E
:1035A00002232A4F03903A681A42FCD12023069343
:1035B000069B5A1E0692002BFAD1254E3368002B2B
:1035C000FCDA0120FFF782FF011E02D0112009B0B2
:1035D000F0BD030003220190009005AD9F2000F094
:1035E000E7FD0321280000F0DBFC02233A681A42C1
:1035F000FCD120230793079B5A1E0792002BFAD178
:103600003368002BFCDA0120FFF760FF0028DDD1D2
:103610000398FEF78BF9AA786B7811041B020B4311
:1036200029780B4363601300113B0A49052B07D827
:1036300001239340A3600B60012323700020C6E7A1
:1036400080231B03F6E7C0469444FF1F90C8004048
:1036500000C800409808FF1F1E4B30B55A68187804
:103660001D4B85B0D31859424B41012100930023D3
:1036700000F05EFB194B1A4A02259A6300221A6574
:1036800010325A658022C4219D65164B1648D2021D
:10369000DA6789004258154B80241A4080231B04A6
:1036A00013434350642341200393E40500F078F969
:1036B000402000F075F96562039D6B1E0393002D99
:1036C000FAD103236362FFF73BFFA562FFF760FFB8
:1036D00005B030BDA044FF1F95FFFEF700C80040B5
:1036E000050001FF04E100E000E100E0FFFF00FF52
:1036F00010B5064B18705960FFF7AEFF002113207C
:10370000034AFFF701FE002010BDC046A044FF1F82
:103710005936FF1FF0B5040085B003920291FEF701
:10372000F1F8882263035B0B52051A438023DB0503
:103730009D6A8023274F0092BA68002601901B03E0
:103740009A420CD9F82326001B041E401C4206D0C6
:103750008022214B52025E6219680A431A60002DD2
:103760000BD100F015FB02221C4B1A608023DB05F5
:103770005A62013A9A6200F0FBFC0023039A9342DA
:1037800020D1002D0AD100F003FB144B03221D6051
:103790008023DB055A629D6200F0EAFC8023BA6850
:1037A0001B039A4208D9002E06D000220A4B0C496E
:1037B0005A621A680A401A600198FEF7B7F80020AA
:1037C00005B0F0BD009A0299D2181278CA5401339C
:1037D000D4E7C0469444FF1F00C8004000C000402A
:1037E000FFFFFEFFF0B587B0029103920400FEF7E1
:1037F00089F8019000F0CCFA802302250122234EA3
:10380000DB0535605D629A6200F0B2FC204F3B68D8
:103810002B42FCD120230493049B5A1E0492002BBC
:10382000FAD11C4D2B68002BFCDA0120FFF74EFE6D
:10383000002802D0112007B0F0BD2000039A0299A1
:1038400000F01EFB022304003A681A42FCD1202338
:103850000593059B5A1E0592002BFAD12B68002B6D
:10386000FCDA0120FFF732FE051EE3D100F090FAEA
:1038700080230322DB0535605A629D6200F078FCEC
:103880000198FEF753F8E0B2D5E7C04600C000400B
:1038900090C8004000C80040F0B5802687B0040002
:1038A000FEF730F8F605B36A02250393029000F0A4
:1038B0006FFA0123244F3D607562B36200F058FC3B
:1038C000224E33682B42FCD120230493049B5A1EC2
:1038D0000492002BFAD11E4D2B68002BFCDA01203C
:1038E000FFF7F4FD002802D0112007B0F0BD200042
:1038F00000F01EFB0223019032681A42FCD1202303
:103900000593059B5A1E0592002BFAD12B68002BBC
:10391000FCDA0320FFF7DAFD041EE5D100F038FAE7
:1039200080230322DB053C605A629C6200F020FC8D
:10393000039B002B01D1FFF703FE0298FDF7F6FF72
:103940006B461879D1E7C04600C0004090C80040DF
:1039500000C8004007B5000201910422000A01A935
:10396000FFF740FF0EBD000073B5050005240B4AAC
:10397000A3005B429B1819686B46DE1D300000F007
:1039800017FB022804D133782B55013CEFD276BDCA
:10399000052CFCD00128FAD10230F8E714090011F7
:1039A0001F2807D8012380228340D20591680B434A
:1039B000936070473F2808D8012380222038834035
:1039C000D20551690B435361F3E75F28F1D8012316
:1039D000802240388340D205116A0B431362E8E726
:1039E0001F2807D8012280218240C9058B68934394
:1039F0008B6070473F2808D8012280212038824000
:103A0000C9054B6993434B61F3E75F28F1D8012265
:103A1000802140388240C9050B6A93430B62E8E776
:103A20001F2810D880230200DB05153A1968012AE7
:103A300006D820229143196019680A431A6070471A
:103A400001228240F6E73F2811D880230200DB05DF
:103A5000353AD968032A06D810229143D960D9682B
:103A60000A43DA60EBE7012220388240F5E75F285D
:103A7000E5D842238022181A413B8340D205516A7F
:103A800099435162516A0B435362D8E710B5040061
:103A9000012813D1A022184992050B685B015B092C
:103AA00013430B60154B164A19681140154A0A4317
:103AB0001A60402219680A431A6010BD0028FCD120
:103AC00001000A2000F044FB21000B2000F040FB25
:103AD000C0220A4B920019680A4340211A601A68F2
:103AE0008A431A60B022044912060B685B015B0925
:103AF00013430B60E1E7C04614F000401CF00040A7
:103B00007F00FEFF80FD010072B6074A1368013393
:103B100013600422054B1A600023054A13608022BB
:103B2000D2055360FEE7C0467808FF1FC0F0004092
:103B3000C4F00040044B054A1A60054B1A6000228D
:103B4000044B1A607047C046140AFF1F841E000011
:103B5000380AFF1FC4F000400023034A1360034AE1
:103B60001360034A1360704754F0004040F1004076
:103B700044F10040002310B5184C8AB00093019323
:103B80002378012B27D06946012000F039F900285D
:103B900017D1009B12490293019B06AA0393114B74
:103BA00002A81B680493104B1B68059300F0C8F92A
:103BB00010220E4906A800F05BF8002804D1FF236C
:103BC000237000200AB010BD0123094A074902A84A
:103BD000237000F0B5F90120F4E7C046BC65FF1F73
:103BE00010290011082900110C29001120290011A9
:103BF000C065FF1F13B501246946012000F000F9DC
:103C0000034B00940193FFF7B5FF200016BDC0469B
:103C1000BB0B000010B5FFF79FFFFFF7EBFF00287D
:103C200002D0024B984710BDFEE7C046E1A200005B
:103C300002B4714649084900095649008E4402BC45
:103C40007047C04602B4714649084900095C490002
:103C50008E4402BC7047C04603B471464908400018
:103C60004900095A49008E4403BC70470000000017
:103C700001B40248844601BC604700BFCD4C01003E
:103C800001B40248844601BC604700BFDD0A010060
:103C900001B40248844601BC604700BF69110100BD
:103CA00001B40248844601BC604700BFF9A6000089
:103CB00001B40248844601BC604700BF894400004B
:103CC00001B40248844601BC604700BFD5440100EE
:103CD00001B40248844601BC604700BF01D7000020
:103CE00001B40248844601BC604700BFC95C0100C2
:103CF00001B40248844601BC604700BFF5350100AD
:103D000001B40248844601BC604700BF6D0B01004E
:103D100001B40248844601BC604700BF053401007D
:103D200001B40248844601BC604700BF71B0000086
:103D300001B40248844601BC604700BFC56D010064
:103D400001B40248844601BC604700BF51B800007E
:103D500001B40248844601BC604700BF61370100DE
:103D600001B40248844601BC604700BF01890000DD
:103D700001B40248844601BC604700BF016C0100E9
:103D800001B40248844601BC604700BF19FA000034
:103D900001B40248844601BC604700BF75A9000019
:103DA00001B40248844601BC604700BF2D6C01008D
:103DB00001B40248844601BC604700BFB70E000052
:103DC00001B40248844601BC604700BFA9D8000086
:103DD00001B40248844601BC604700BFF5B0001141
:103DE00001B40248844601BC604700BFE90B0100F2
:103DF00001B40248844601BC604700BF156B010056
:103E000001B40248844601BC604700BFE1AC000039
:103E100001B40248844601BC604700BFE9F60000D7
:103E200001B40248844601BC604700BFA1AF000056
:103E300001B40248844601BC604700BFC1F70000DE
:103E400001B40248844601BC604700BFADAE00002B
:103E500001B40248844601BC604700BF8B52010098
:103E600001B40248844601BC604700BF4DF9000020
:103E700001B40248844601BC604700BF21440000F1
:103E800001B40248844601BC604700BF957301003D
:103E900001B40248844601BC604700BFF9ED000050
:103EA00001B40248844601BC604700BF791201009A
:103EB00001B40248844601BC604700BF7997000006
:103EC00001B40248844601BC604700BFE9270000F6
:103ED00001B40248844601BC604700BF016701008D
:103EE00001B40248844601BC604700BFEDA5000054
:103EF00001B40248844601BC604700BF8914010038
:103F000001B40248844601BC604700BF8937010004
:103F100001B40248844601BC604700BFDD0C0100CB
:103F200001B40248844601BC604700BFB35201009F
:103F300001B40248844601BC604700BFA96F01007C
:103F400001B40248844601BC604700BFDD3F000069
:103F500001B40248844601BC604700BF8D82000066
:103F600001B40248844601BC604700BFE917010064
:103F700001B40248844601BC604700BF85C100000F
:103F800001B40248844601BC604700BF090E00002E
:103F900001B40248844601BC604700BF1907010014
:103FA00001B40248844601BC604700BF3D71010076
:103FB00001B40248844601BC604700BF913800113B
:103FC00001B40248844601BC604700BF9D6A0000FE
:103FD00001B40248844601BC604700BFC9A9000083
:103FE00001B40248844601BC604700BFBD0B01001C
:103FF00001B40248844601BC604700BFE94C01009F
:1040000001B40248844601BC604700BF75F8000057
:1040100001B40248844601BC604700BF116E000035
:1040200001B40248844601BC604700BFE9D40000E7
:1040300001B40248844601BC604700BFE51201009C
:1040400001B40248844601BC604700BF0D52010024
:1040500001B40248844601BC604700BFC11501009D
:1040600001B40248844601BC604700BFF935010035
:1040700001B40248844601BC604700BF5976010084
:1040800001B40248844601BC604700BF090E00002D
:1040900001B40248844601BC604700BFC1A50000CE
:1040A00001B40248844601BC604700BF851201008C
:1040B00001B40248844601BC604700BF6DF60000B1
:1040C00001B40248844601BC604700BF09340100C6
:1040D00001B40248844601BC604700BFCD0C01001A
:1040E00001B40248844601BC604700BF855201000C
:1040F00001B40248844601BC604700BF21A900000A
:1041000001B40248844601BC604700BFBD5C0100A9
:1041100001B40248844601BC604700BF013401007D
:1041200001B40248844601BC604700BFF90D01009C
:1041300001B40248844601BC604700BFED6B01003A
:1041400001B40248844601BC604700BFC16601005B
:1041500001B40248844601BC604700BFE59C0011E1
:1041600001B40248844601BC604700BF53B9000057
:1041700001B40248844601BC604700BF9DA900000D
:1041800001B40248844601BC604700BFED680100ED
:1041900001B40248844601BC604700BF8D11010094
:1041A00001B40248844601BC604700BFD9B000009A
:1041B00001B40248844601BC604700BF496D01005C
:1041C000020000000ABA001101000000D8B7001177
:1041D0000200000006BA0011010000000042FF1FAB
:1041E00002000000E0B70011010000000463FF1F9F
:1041F0000200000004BA0011030000007862FF1FF3
:1042000012000000020000000ABA001101000000C4
:1042100020B800110200000006BA001101000000E1
:104220001DB80011020000002AB8001103000000B0
:10423000B362FF1F0200000004BA00110300000077
:10424000C862FF1F0200000006BA00110100000052
:104250001CB800110200000028B800110300000083
:104260008962FF1F0200000004BA00110300000071
:10427000AA62FF1F020000000ABA0011010000003C
:1042800064B800110200000006BA0011010000002D
:104290004943FF1F0200000076B800110100000032
:1042A0005BB800110200000006BA00110100000016
:1042B0004843FF1F0200000074B800110100000015
:1042C000D062FF1F0200000006BA001101000000CA
:1042D0004743FF1F0200000072B8001101000000F8
:1042E0004BB800110200000006BA001101000000E6
:1042F0004643FF1F0200000070B8001101000000DB
:1043000046B800110200000006BA001101000000CA
:104310004543FF1F020000006EB8001101000000BD
:1043200041B800110200000006BA001101000000AF
:104330004443FF1F020000006CB8001101000000A0
:104340003CB8001102020202020200002D4A0011D4
:10435000294A0011B8B80011900118001800FFFF99
:104360000701020304050602010600000000000028
:10437000000000000000000000000000000000003D
:104380000000000000000300020000000ABA001153
:104390000100000038B900110200000006BA001147
:1043A00001000000F843FF1F0200000042B90011A5
:1043B00001000000FE62FF1F0200000004BA0011AD
:1043C000030000006C65FF1F0200000006BA001128
:1043D00001000000F843FF1F0200000040B9001177
:1043E000010000000063FF1F0200000004BA00117A
:1043F000030000006465FF1F1200000000010000C0
:1044000000000111FFFF0000504859360000000075
:104410000000000001000000C9B800110B000500F9
:10442000F7000000B4000028002800283075A00024
:10443000A000A000A00000080008E001F0001000AB
:10444000100010001000100010005000500050002C
:1044500010001000D0070000000000000F00010055
:104460000500307507001000010081FF000000000A
:10447000FF000000BD6E0011C56C0011556A0011EF
:10448000FFFF0100FF000000D998001155960011B0
:104490006D95001100000000000000000000080001
:1044A000040000003B0001085902E00188212800B7
:1044B000FF000000020000000ABA00110100000025
:1044C000D0BA00110200000006BA0011010000007D
:1044D0003145FF1F0200000002BA00110100000078
:1044E0007869FF1F0200000006BA001101000000F9
:1044F0003045FF1F0200000000BA0011010000005B
:104500002E45FF1F0200000006BA00110100000046
:104510002C45FF1F02000000FEB900110100000041
:104520002445FF1F1800180000009001020000033E
:1045300002020000020000000ABA0011010000009F
:10454000E4BA00110200000006BA001101000000E8
:104550007445FF1F02000000FCB9001100000000BC
:10456000000000000200000004BA00110300000077
:064570009869FF1F20FF07
:040000051FFF184180
:00000001FF
